:020000022000DC
:1060000000000120756302005D6302005F6302000F
:106010006163020063630200656302000000000028
:1060200000000000000000000000000067630200A4
:1060300069630200000000006B6302006D630200F0
:10604000819B02006F63020091A102006F63020056
:106050006F6302006F63020045A0020061A20200AC
:106060006F6302006DA802006F630200ADA1020021
:106070006F6302006F6302006F6302006F630200D0
:1060800025AA02004D7602006F6302006F630200D2
:106090006F6302006F630200B9E002006F630200E9
:1060A0006F6302006F6302006F6302006F630200A0
:1060B0006F6302006F630200000000000000000038
:1060C0006F6302006F6302006F6302006F63020080
:1060D0006F6302006F6302006F6302000000000044
:1060E00000000000000000000000000000000000B0
:1060F00000000000000000000000000000000000A0
:10610000000000000000000000000000000000008F
:10611000000000000000000000000000000000007F
:10612000000000000000000000000000000000006F
:10613000000000000000000000000000000000005F
:10614000000000000000000000000000000000004F
:10615000000000000000000000000000000000003F
:10616000000000000000000000000000000000002F
:10617000000000000000000000000000000000001F
:10618000000000000000000000000000000000000F
:1061900000000000000000000000000000000000FF
:1061A00000000000000000000000000000000000EF
:1061B00000000000000000000000000000000000DF
:1061C00000000000000000000000000000000000CF
:1061D00000000000000000000000000000000000BF
:1061E00000000000000000000000000000000000AF
:1061F000000000000000000000000000000000009F
:10620000354936480A1A02D0072291438D4634494F
:1062100034480A1A06D00722914381F309880222E2
:1062200082F3148830483149314A00F044F831484B
:106230003149324A00F03FF831483249324A00F0E1
:106240003AF832483249334A00F035F83248334997
:10625000334A00F030F833483349344A00F02BF821
:1062600033483449344A00F026F83448344900228F
:1062700000F02CF833483449002200F027F8334866
:106280003349091A082902DB002202604160314AC1
:1062900090471F481F49884205D00268043003B464
:1062A000904703BCF7E700208646EC46002000211B
:1062B000294A9047FEE7884207D0521A05D0037852
:1062C00001300B700131013AF9D17047884202D098
:1062D00002700130FAE770470000012000E0002062
:1062E0000000012000000120D8050300EC2A002056
:1062F0004C2B0020D0630200D06302009AEA020017
:10630000D8050300EC2A0020EC2A0020FCEB020058
:10631000FCEB0200FCEB0200FCEB0200FCEB0200D9
:10632000FCEB0200FCEB0200FCEB0200D6050300D4
:10633000380603004C2B00204C2B00204C2B002057
:106340005843002058430020584300205843002061
:10635000586300209D63020049BD0200FEE7FEE78E
:10636000FEE7FEE7FEE7FEE7FEE7FEE7FEE7FEE705
:1063700000F002B8FFF7FCBF0F484FF00701884359
:1063800085460E4880470E48016841F4700101605F
:10639000BFF34F8FBFF36F8FFFF732BF09480A4932
:1063A0000A4A884207D0521A05D0037801300B7090
:1063B0000131013AF9D170470000012039960200FD
:1063C00088ED00E0E8EB0200D82A0020EC2A00204B
:1063D0007047000007B5044B0093044A402300F0C7
:1063E00032F803B05DF804FBF16302004D2B00208E
:1063F0002DE9F84388461446B2B10F4B0F4E0325E2
:10640000002743F00109224608EB0701002006F0AF
:10641000C5FA0744241A48B933782BB14FF47A40AF
:10642000C847013D02D13570BDE8F88301233370C0
:10643000002CE8D1F8E700BF00EC02004C2B002054
:10644000704706F0DBBAF0B595B01D461646084613
:106450000C4601F0CDFC1A9B0D93CDE90865002593
:106460002B46082205A920460A958DF82C500C953C
:1064700001F0DAFC079B0293069B03939DF814300E
:106480008DF8115003F00302012A1DD1BDF814202C
:10649000059DC3F3C203C2F383168DF81030B2001A
:1064A00008230EA9204601F0BFFCC5F3952508ABD3
:1064B0000093324602AB0EA9284600F03BFB204673
:1064C00001F09AFC15B0F0BD022AF8D1BDF81650C3
:1064D000C3F3C203C5F389158DF810300827082DC2
:1064E0002E4628BF08263B4632460EA9204601F01C
:1064F0009BFCAD1B08AB02AA31460EA8374400F046
:106500007DFB002DEBD1DAE708B5FFF79AFF0448D1
:10651000042100F079FA034B01225A7108BD00BF33
:10652000D8EB0200EC2A0020037813F0040216D006
:1065300003F00303012B03D0022B09D00120704785
:106540000A6800880232C0F3831002440A60F5E74B
:106550000B684288023303EB92130B60EEE71046A0
:10656000704700002DE9F04FDFF81CA187B00F46FF
:1065700000230446861C0DF1070015468DF80730F0
:1065800000F0F6FEDAF804203A60DAF8083003F595
:1065900080739B1A0AF21C470AF583690AF21448B1
:1065A000B3421AD30020002D69D004F00F039B01E1
:1065B00043F0050363F30F00DAF80430DAB2033274
:1065C00033444AF822009DF80700CAF8043000F06E
:1065D000F3FE012007B0BDE8F08F0121384601F03D
:1065E0004CF9484601F064F9404601F061F9DAF8E7
:1065F00008000290C0B203300AEB800002A9FFF746
:1066000093FF029B30BBDAB20AEB8202D16803919E
:106610009A1C0133DBB20AEB83030292D3F80CB06D
:1066200001F00303012B22D0022B15D083464046F4
:1066300001F041F910B1029BCAF8083059463846BA
:1066400001F01BF9DAF80830DAF8042003F580735A
:106650009B1AA5E7D8B2CEE7BDF80E30C3F3891375
:1066600003334FEA1B4B02EB93030293DFE7BDF8C2
:106670000C30C3F383134FEA1B4B1344F5E7A40517
:1066800044F0060098E700BF602C0020064B074846
:1066900010B500221A7001F064FB044610B90448DA
:1066A00001F00CFC204610BD602C002014EB020011
:1066B0003CEC020030B50A4C71B10A4A0A49121B7F
:1066C000D20800239A4201D1002030BD31F8235076
:1066D000854202D00133F5E7034654F83300F4E76E
:1066E00028EB0200D8EB0200EC2A0020094B01390C
:1066F00003EBC000032909D8DFE801F00A02040611
:106700000420704700797047407970470020704737
:106710000220704728EB0200034BD3E90130C31A73
:1067200058425841704700BF602C00202DE9F041CD
:1067300086B0FFF7F1FF0546002840F0ED80774C6A
:10674000C4F81804BFF34F8FA3680293DBB203337E
:1067500004EB830002A9FFF7E7FE029B18B1D4F80F
:106760001824002A5AD0DAB2991C013304EB8202B1
:10677000DBB204EB8303D268DB68049302F003030B
:10678000022B0392029154D1BDF80E306448C3F33A
:106790008917502F3E4628BF502606F1080166F3A0
:1067A0008F13C1F30901ADF80E3001F0F2FA05467E
:1067B000002800F09C8001F01BFB0023082203A9A5
:1067C000284601F027FB0299CB43DBB20133C9B263
:1067D0000331B6EB830F4FEA830204EB810125D925
:1067E0005FFA82F80823A6EB0806284601F012FBA0
:1067F000F6B208F108034B4903F0FC033246284681
:1068000001F008FB029B033703EB97070297D4F8CC
:106810001834002B43D1D4F8106453E062689A42D4
:1068200094D8A260284606B0BDE8F081082332461D
:10683000E5E7012B5BD1BDF80C303948C3F3831178
:10684000062928BF062161F38913023101F00F01E7
:106850008900ADF80C3001F09CFA0546002846D0BE
:1068600001F0C6FA0023082203A9284601F0D2FA53
:106870000026BDF80C20C2F38312B300964203F148
:106880000803C4D202994A1CC9B20331029204EB34
:1068900081010422284601F0BDFA0136E9E72846C5
:1068A00001F0AAFAFFF738FF80F00100C5B2B9E79E
:1068B000F3685B7923B1336829461B6830469847F3
:1068C000F3681E68002EF3D1284601F095FA0DF109
:1068D00007008DF8076000F04BFDD4F818340BB9B1
:1068E000029BA3609DF8070000F066FDDAE7D4F88C
:1068F000104454B90C4B0D480D49C01AC00800048F
:1069000040F0020000F05CF8CCE7236820469B686A
:106910009847E3681C68ECE7002583E7602C0020BB
:1069200014EB02006C2C002028EB020078EB020034
:1069300024EC02002DE9F34704460E46924601A9D5
:10694000012218469946FFF70DFE1B4F10B3019D1B
:106950004FF00008AA1CC84508EB020123D11748D4
:10696000002100F043FF80F31000000440EA1440CF
:10697000E4006B1C04F03804DBB2EDB244F0010417
:1069800007EB8303033544EA881444EA8624D8607D
:1069900047F825403B781BB1FFF7C8FE0028FBD124
:1069A00002B0BDE8F087C9B207EB81015AF8283080
:1069B000CB6008F10108CEE7602C00207C3000207D
:1069C00000231A46FFF7B6BF07B50123019201AABB
:1069D000FFF7B0FF03B05DF804FB07B5CDE9002376
:1069E00002236A46FFF7A6FF03B05DF804FB1FB55C
:1069F000CDE90123069B039301AA0323FFF79AFF26
:106A000005B05DF804FB000030B50F4CD4F810243D
:106A100003460020114631B9D96808714AB9C4F853
:106A200010340A6030BDC9680D79854206D0096806
:106A3000F1E7D26814680C601360F3E701300A28AC
:106A4000E8D14FF0FF30EDE7602C002038B5084B5F
:106A50000125D3F810441D7004B938BDE3685D7199
:106A6000236820465B689847E3681C68F4E700BF2A
:106A7000602C002030B5C38885B004460D4633B184
:106A8000144A00921449154A284601F07CFD217AE7
:106A900005291DD0637A4BB1A088FFF727FE104B64
:106AA000104953F82020284601F06DFD227A0E4B44
:106AB000A08853F8222003920021FFF7FBFD039AE0
:106AC0000A490346284605B0BDE8304001F05BBDE9
:106AD00005B030BD68EC020050EC020048EC02004A
:106AE000D4EC02006DEC0200F8EC020070EC020045
:106AF00007B503460846197A052911D05B7A2BB1F0
:106B0000094A0A49019001F03EFD019808490190A7
:106B100001F039FD019803B05DF804EB01F028BDE8
:106B2000002AF8D0F2E700BF68EC02006DEC02002A
:106B30004EF702002DE9F04385B01F460C9D00235F
:106B400095F80C902B7306460C469046294638461D
:106B5000FFF790FFB8F1060F09D8DFE808F004123C
:106B6000181F283340003146284601F00CFD002252
:106B700029463846FFF7BCFF85F80C9005B0BDE804
:106B8000F08322683146284601F0FDFCEFE7D4E9A6
:106B900000233146284601F0F6FCE8E7A36800939D
:106BA0003146D4E90023284601F0EDFCDFE7E36835
:106BB0000193A36800933146D4E90023284601F0ED
:106BC000E2FCD4E723690293E3680193A36800938E
:106BD0003146D4E90023284601F0D5FCC7E76369B4
:106BE000039323690293E3680193A36800933146FA
:106BF000D4E90023284601F0C6FCB8E708292DE9AE
:106C0000F74F80460E4617461C463DD800251B7B95
:106C10002573214610460193FFF72CFFDFF88CA067
:106C2000DFF88CB0AE4232D918F80520594620461C
:106C300001F0A9FC0135082DF4D11B49DFF874A03F
:106C4000DFF874B0204601F09EFC4FF000094E457D
:106C500024D918F809507E2D1ED8284607F06AFE60
:106C6000002814BF2A462E225946204601F08BFCEC
:106C700009F10109B9F1080FE9D10122214638468D
:106C8000FFF736FF019B237303B0BDE8F08F514639
:106C9000204601F078FCCDE72E22E5E7514620465C
:106CA00001F071FCE4E700BF84EC020080EC02001C
:106CB0007AEC020082EC020086EC0200C30710B5F9
:106CC00007D4F023054A4008145C234019431154AB
:106CD00010BD0901C9B20F23F4E700BF48310020FD
:106CE00030B5094B1C78094B196800239C4202DC23
:106CF0000022104630BD11F83350854201EBC3022B
:106D0000F7D00133F2E700BF1831002058310020DE
:106D100013B504460191FFF7E3FF38B143682BB187
:106D20000199204602B0BDE81040184702B010BDDE
:106D3000034B044819680022490800F02CBA00BF30
:106D40001C3100202031002010B5C0B2FFF7C8FF71
:106D50000446007803F06CF963785A1E534253419D
:106D6000834208D1044BD3E90023134303D1BDE888
:106D70001040FFF7DDBF10BD4031002037B543089C
:106D8000374AD35CC2074CBF1B0903F00F0304460C
:106D90000D46042B25D8DFE803F003262F3C4000E6
:106DA000F9B10121FFF78AFF00230DF107008DF8EB
:106DB000073000F0DDFA0120A4F12003C4F1200126
:106DC000284A20FA01F100FA03F30B43A040D2E96C
:106DD000004120430B43C2E900039DF8070000F087
:106DE000EBFA03B030BD002918BF0221204603B0E2
:106DF000BDE83040FFF762BF49B10321FFF75EFFF6
:106E00000121204603B0BDE83040FFF781BF0121DA
:106E1000ECE70029E5D10421E8E709B10321E5E722
:106E2000FFF74CFF29462046FFF772FF0DF10700E0
:106E30008DF8075000F09CFA0120A4F12003C4F162
:106E40002001084A20FA01F100FA03F30B43A040A5
:106E5000D2E9004124EA000021EA0303BBE700BFB6
:106E600048310020403100202DE9F041124E134FEF
:106E700000243378A34208DC114BD3E900231343E9
:106E800018D0BDE8F041FFF753BF3D6805EBC408DB
:106E900015F8340003F0CCF898F801305A1E53422C
:106EA0005341181A4142414115F83400FFF766FF7B
:106EB0000134DEE7BDE8F0811831002058310020B0
:106EC00040310020092AF7B505460C4616463ED942
:106ED00002F0EEFEE8B11F4B1F481D601F4B204F14
:106EE0001C70204B002110221E6007F051FD1E4B2C
:106EF00000200021C3E90001013CE4B20326FF2C7D
:106F00000DD11A4A1A48002103B0BDE8F04000F044
:106F100037B902F095FE0028DDD003B0F0BD9DF832
:106F2000063015F834008DF8046005EBC40223F038
:106F300007038DF8063001A993788DF805303A469D
:106F400002F0B8FF013CE4B20028D8D0E5E7072002
:106F5000E3E700BF583100204831002018310020FD
:106F6000496D02001C31002040310020696E020092
:106F700018ED020070B5084D084E00242B789C4295
:106F800001D3002070BD3368012113F8340003F0F1
:106F900009F80134F2E700BF183100205831002011
:106FA0001FB50021039001AA44F20100CDE90111AF
:106FB00000F004F805B05DF804FB000038B572B6C7
:106FC000FFF744FDFFF7B2FB0028FBD1104B114C3B
:106FD000114D1249E41AE408240444F00100FFF7BB
:106FE000EFFCD5F8F030DB0700D500BE0C4944F0CB
:106FF0000200FFF7E5FCBFF34F8FEA68094B02F48C
:10700000E0621343EB60BFF34F8F00BFFDE700BFAB
:1070100028EB020078EB020000ED00E01CED02001E
:1070200028ED02000400FA0510B5D0E90243D1E9C9
:107030000202A04272EB03032CBF0120002010BD0E
:1070400008B50A4800F0EBFA094AD2E90031C01845
:10705000084BD3E9002341F10001904271EB030397
:1070600003D210F1807041F1000108BDF42A002024
:1070700060310020D831002037B505460C460A485B
:1070800001A900F022FB60B10570446001A9064827
:1070900000F045FB18B1054800F0C6FA002003B027
:1070A00030BD0420FBE700BFC4310020F42A0020DB
:1070B00038B5184B1B78044613B90025284638BD4F
:1070C0000028FAD0037F03F0FF05002BF5D0FFF76F
:1070D000B7FFD4E90223904271EB030314D3236971
:1070E00003B92377D4E90530984721690029E4D012
:1070F000237F03F0FF05002BDFD0D4E902325B18B9
:1071000042F10002C4E902320348214600F0F5FED4
:10711000D4E700BF6831002044ED020013B5114BE5
:1071200011491868019008231048582200F098FA75
:10713000044698B90E4A0F4801A900F061F90446C7
:1071400060B90C48012100F04DFA01230A4A0948B0
:10715000194600F0AFF9094B01221A70204602B01F
:1071600010BD00BF40ED02006C310020C431002092
:10717000E1710200F42A0020FFFF7F006831002047
:107180003AB103685A614A1E5142514119610020C7
:1071900070470720704738B5037F04460D4683B912
:1071A0008261FFF74DFF2369281841F10001C4E90E
:1071B000020103B1256121460020BDE83840FFF7F8
:1071C0005BBF002038BD0023014603770120FFF795
:1071D00053BF0000014800F022BA00BFF42A00208B
:1071E0002DE9F347064600F005FA40B1584AD2E9C6
:1071F000003113F1807341F10001C2E90031002137
:10720000304600F006FA38B1524C236823B12068AA
:10721000FFF74EFF002323600121304600F0F9F90B
:1072200020B1FFF70DFF4C4BC3E900014B48494D1E
:107230004B4C4C4F01A900F082FA002842D1DFF8F4
:107240002081444CDFF82491404600F06CFE236816
:10725000002872D07BB12368D0E90252D3E902132F
:107260008D4272EB03032AD223681B7F1BB1216876
:10727000404600F042FE404600F04FFED0E9027A60
:107280000546FFF7DDFE381A6AEB010A01287AF19C
:10729000000345DBB0F5350F40D3FFF79BFF324AC3
:1072A00002444FF496030021484600F023F90028D9
:1072B0003ED1236813B9304600F0F4F8256002B0DF
:1072C000BDE8F0870378012B1DD0022B09D14FF0C8
:1072D0000008204600F021FE002836D080F81C80EF
:1072E000F7E73BB941680B7F23B901230B772046B1
:1072F00000F003FE01A9194800F04CFA01A9174853
:1073000000F01DFA99E741682B68994202D10023E9
:107310002B60EFE7204600F009FEEBE7AA68C0E724
:107320000021484600F06BF92846FFF7C1FE01E056
:107330000D28F9D00023236086E7002BBFD130460B
:1073400002B0BDE8F04700F0B1B801233B70D1E7CF
:1073500060310020E0310020D8310020C43100200D
:1073600044ED020068310020FFFFB400F42A002041
:1073700070B5EFF3108672B60C4A946801239CB97D
:1073800093600B4B0B4DD3F8801029401160C3F86C
:107390008050D3F8841051604FF0FF32C3F884203E
:1073A000047006B962B670BD0370FAE7E4310020DC
:1073B00000E100E0FC06FFBD084B9A6810B55AB129
:1073C00050B9EFF3108172B6054A1C6814605C680E
:1073D0005460986001B962B610BD00BFE43100206E
:1073E00000E100E0435882B03BB1002343504358D2
:1073F0000193019B012002B070471846FBE7000093
:10740000F8B5204B4479204E43F824201F4A204BE6
:1074100006EBC4049B1A2279DB081B0432B143F04B
:1074200002001C49FFF7CCFA0820F8BD02680C885E
:10743000C2F8084590F904508A7804795201002D69
:10744000D2B219DB14494F1987F8002301226D09C4
:1074500004F01F0402FA04F441F82540427906EBD7
:10746000C201012446F832000C7143F003000B49BD
:10747000FFF7A6FA0020D8E7094904F00F040A55DF
:10748000ECE700BFF8310020F031002028EB0200CB
:1074900088EB020050ED020000E100E072ED020016
:1074A00014ED00E0036801221A60704703680122AE
:1074B0005A60704773B501F15005AD000068ADB278
:1074C0004FF480348C400026C0F80843C0F848438D
:1074D000465101F5A8714559019522F07F42019D61
:1074E00040F82120C0F844430BB1C0F8044302B077
:1074F00070BD00002DE9F74F0D4622F07F44026871
:107500004FF4803705F150068F408046B60002EBFD
:107510008500C2F84873B6B2C2F80873D2F80415F1
:1075200099464FF0000BD0F84035C0F8401542F8AE
:1075300006B05B1A9259009223F07F43012B009A08
:107540004FEA850A0CD1264B4FF4806043F00103CB
:107550009847D8F8003043F806B09B590193019B37
:10756000D8F80010D1F80465C1F84473A31B23F0C8
:107570007F43012B1CD11A4B05F5A875013443F04C
:10758000010341F825404FF480609847D8F8003057
:10759000D3F804359E4209D1D8F800300020C3F852
:1075A0004473C3F8047303B0BDE8F08F0D20FAE70D
:1075B0008A44C9F1FF13CAF84045D1F80405221ADC
:1075C000013A22F07F4203F57F439342EED3002A33
:1075D000E2D10134CAF84045D1F804359842DAE7DF
:1075E00090ED020003680222C3F8442309B1C3F8F6
:1075F0000423704700684FF48271FFF7F3BE4FF425
:10760000803303FA01F10368C3F84813C3F8081381
:10761000704750318900006889B2FFF7E3BE036804
:10762000D3F804057047000090F90430002B09DB03
:107630005A09012103F01F0301FA03F34032024902
:1076400041F82230704700BF00E100E0024B034ADE
:107650001B681068184700BFF8310020F031002087
:1076600010B561B1B2FBF3F403FB1424A4B244B926
:10767000C0E9001484608281C381204610BD0E20C1
:10768000FCE70920FAE782B050E8022FC188B2EB8C
:10769000324F4FF0000317BF92B241EA014142EA74
:1076A000014104E04268B2EB324F08BF012340E8D9
:1076B0000212002AE8D18DF807309DF80730002B20
:1076C0000CBF1120002002B0704737B550E8013FD1
:1076D0009DB2C48925448489A54228BF2D1B0489F5
:1076E000A54202BFBFF32F8F002207E0C5EA0305C2
:1076F00040E80154002CE9D14FF001028DF803203D
:107700000193019A0A609DF8031001F0FF0321B173
:10771000006810FA82F003B030BD1846FBE70A8813
:107720004B889A4209D150E8012FC2EA024240E850
:107730000123002BF7D1012070470020704737B597
:1077400050E8023F1FFAA3F5C488A54202BFBFF369
:107750002F8F00220DE0C48925448489A54228BFCB
:107760002D1BC3EA054540E80254002CE8D14FF038
:1077700001028DF803200193019A0A609DF803101D
:1077800001F0FF0321B1006800EB124003B030BDEF
:107790001846FBE70A884B889A4209D150E8022F25
:1077A000C2EA224240E80223002BF7D101207047B1
:1077B0000020704701F01F024B090121914000EBAE
:1077C000830000F02AB801F01F0301229A404B0900
:1077D00000EB8300D14300F038B84B0901F01F01E2
:1077E00050F82300C84000F00100704710B5034670
:1077F00053E8000F0A4643E8002494F0000FF7D145
:1078000010BD10B5034653E8000F40EA010243E8FB
:10781000002494F0000FF6D110BD10B5034653E8D4
:10782000002F42EA010043E8000494F0000FF6D173
:1078300010BD10B5034653E8000F00EA010243E80B
:10784000002494F0000FF6D110BD10B5034653E8A4
:10785000002F02EA010043E8000494F0000FF6D183
:1078600010BD10B5034653E8000F00EB010243E8DA
:10787000002494F0000FF6D110BD10B5034653E874
:10788000002F02EB010043E8000494F0000FF6D152
:1078900010BD10B5034653E8002FA2EB010043E8EA
:1078A000000494F0000FF6D110BD0121FFF7A9BF2D
:1078B0000121FFF7B2BF0021FFF7BBBF10B590B1A8
:1078C000D0E9012301689B1ADBB20A60013BDBB2FD
:1078D000FF2B026802D10020107110BD11684C1CF2
:1078E00014600B70F2E70E20F7E737B50546002469
:1078F0000DF107008DF80740FFF73AFD2A686B6825
:10790000116899420ED9481E106011F8013CEC68CC
:10791000298A01FB0344AB6811791B1ADBB2994237
:1079200038BF13719DF80700FFF746FD204603B0EE
:1079300030BD37B5054600230DF107000C468DF824
:107940000730FFF715FD2A681368591C1160E968B4
:10795000641A298AB4FBF1F41C709DF80700FFF744
:107960002BFD03B030BD0A2938B504460D4602D1BF
:107970000D21FFF7F8FFA3682268591CA160D554B8
:10798000D4E901329A4204D32046BDE8384000F0E1
:10799000EFBD38BD2DE9F84F9846DDE90A4315469D
:1079A00082460F460A464FF00109AA420FD2C1454E
:1079B00038BFC14613F0010B01D16CB90024012678
:1079C000B8F1010F1BD908F1FF386E43F8E709F150
:1079D0000109B2FBF5F2E8E79B070ED5B8F1000FFD
:1079E0000CBF30262026A145E9D2013C3146504645
:1079F000FFF7B9FF002CF6D1E0E72026F3E7B7FB4D
:107A0000F6F39D42E1D9DFF83C80B7FBF6F3504630
:107A100018F8031006FB1377FFF7A5FF3346AB42B8
:107A2000B6FBF5F6F1D2BBF1000F02D00CB1A145C7
:107A300001D3BDE8F88F20215046013CFFF793FFAA
:107A4000F4E700BF96ED02002DE9F74F0546174613
:107A50008846002900F03E8118F8011B49B92B7BAC
:107A6000002B00F03781284603B0BDE8F04F00F04E
:107A70007FBD252940F0B780002698F800302D2BD7
:107A8000424608F1010823D0302B24D02B2B25D0DF
:107A900000242A2B02F1010123D13B681A1D1B6827
:107AA0003A601C440A4613782E2B26D101324FF03F
:107AB000000A104610F8011BA1F1300CBCF1090FAF
:107AC0001DD80A2303FB0A13A3F1300A0246F0E78C
:107AD00046F00106D1E746F00206CEE746F004067E
:107AE000CBE711F8013CA3F130000928DBD80A22CA
:107AF00002FB0434303C0A46CBE74FF0000A12F890
:107B0000011B01F0FB0068289046F8D0782909D8BD
:107B10006F290CD8632962D022D8252963D058292F
:107B200000F0888098F80030002B95D197E77039E5
:107B30000829F7D801A353F821F000BFAF7C020059
:107B4000257B0200257B0200457C0200257B02008C
:107B5000237C0200257B0200257B0200357C02008D
:107B6000642901D06929DDD13A68D2F80090111D4D
:107B700089EAE9723960A2EBE9724FF0010B092A38
:107B800035DCD34538BFD3462CB1B9F1000F01DB4A
:107B9000720700D5013CB30702D5BAF1000F03D03C
:107BA000F00701D44CBB0024B9F1000F2DDAC9F164
:107BB00000092D212846FFF7D6FE06F00302022A0F
:107BC00004D1BAF1000F01D11CBB0024CDE900465D
:107BD00053460A2249462846FFF7DCFEA2E73B68E7
:107BE0001A1D19783A602846FFF7BDFE9AE70A2366
:107BF0000BF1010BB2FBF3F2C1E7A345D4D2202174
:107C00002846013CFFF7AFFECCE77107D5D52B2105
:107C1000D0E7A345DAD230212846013CFFF7A3FE86
:107C2000D2E73968CDE900460A1D3A6053460A2278
:107C30000968D0E739680A1D3A60CDE90046534625
:107C40001022F5E73B681A1D3A6016F00106D3F8DA
:107C5000009024D1B9F1000F03D0484606F0EDFEA4
:107C60000646B4421DD809F1FF3919F8011F002951
:107C70003FF458AF2846FFF776FEF6E72846013670
:107C8000FFF771FE19F806100029F7D1A642BFF4DC
:107C900049AF20212846013CFFF765FEF6E70026A4
:107CA000F0E720212846013CFFF75DFED9E73B685D
:107CB0001A1D3A60302128461C68FFF754FE7821CF
:107CC0002846FFF750FE00220823CDE90032214666
:107CD000102280E703B0BDE8F08F00BF2DE9F84F18
:107CE000B0F806A04579D2F800B09DF828900AFBBC
:107CF00005F5043D88460BEB0301A94203F104049A
:107D000088BFA5EB030BB4FBFAF607460AFB164443
:107D1000C2F800B04EB9AAEB04055D4528BF5D4628
:107D2000BBF1000F04D1BDE8F88F3F68013EF1E7D9
:107D3000043408EB06003C442A46B9F1000F0DD08C
:107D40002146ABEB050B06F0FAFDDA452E443F6801
:107D500055464FF0000428BF5D46E1E70146204646
:107D6000EFE7FFF7ABBDF8B546790146721E054651
:107D7000002393422D6803D30024A64202D8F8BD05
:107D80000133F6E70F682846FFF7D3FD0134394683
:107D9000F3E72DE9F843068ACD1C0746FFF7A5FD5A
:107DA000043E35440446B5FBF6F5F0B14FF480735C
:107DB000EDB28380C680013D076081464FF0000828
:107DC000A84512D23846FFF790FD064648B16379C0
:107DD0000133637108F10108C9F8000007608146AA
:107DE000EEE72046FFF7BFFF34462046BDE8F883A4
:107DF00001210430FFF741BD10B5012104460430D4
:107E0000FFF747FDC0B220B92046BDE81040FFF79C
:107E1000AABF10BD1FB503920022009203AAFFF76C
:107E20005DFF05B05DF804FB1FB5039201220092CF
:107E300003AAFFF753FF05B05DF804FB41DF70476D
:107E4000064B10B500241C70054B1C60BFF35F8F00
:107E50000449054800F03BF8204610BD04320020DC
:107E600008320020B0ED0200FC31002007B50023ED
:107E70000DF107008DF80730FFF77AFAF1EE103AAE
:107E800023F09F03E1EE103ABFF35F8F0A4B4022CD
:107E9000C3F884219DF80700FFF78EFA06F0F2F888
:107EA00020B103B05DF804EBFFF7C8BF20BF40BFAF
:107EB00020BF03B05DF804FB00E100E0836800220E
:107EC0005A60C3E904229A60DA601A6070470B684E
:107ED0004A684360934208BF0023016008BF4360C3
:107EE0007047436843B10268916852680B449342FB
:107EF000436004BF00234360704770B54468064682
:107F00000D46206818B1B3682946984718B9236808
:107F10002B60256070BD2468F3E74368186808B1DA
:107F200002681A60704743681868704743681868A9
:107F300000B97047884203D102681A600120704777
:107F400003460068F4E7000010B50D49A1F59472EE
:107F5000914201D800200FE08C1AE30F03EBE403F9
:107F60005B1002EBC30452F83330834205D802D2CF
:107F700004F10802ECE7606810BD2146E8E700BFA5
:107F8000BCF2020008B5FFF7DFFF024B002808BF74
:107F9000184608BD7FF102002DE9F8430468054644
:107FA00094F8200002F0C0FC04F11807FF264FF0FF
:107FB000FF394FF00008207AFF2802D002F0B4FC0D
:107FC0002672607AFF2802D002F0AEFC667220684A
:107FD000431C03D001F0D8FEC4F8009084F80B8055
:107FE0000C34BC42E7D16868BDE8F84302F0C2BB7C
:107FF0002DE9F041134EDFF850800C460025012793
:1080000006EB4106735D5BB1735D013BDBB27355FB
:10801000735D93B958F824301B682046DB69984794
:108020004DB167B1084B53F824300221BDE8F0414F
:10803000586802F012BC0125E4E70027F0E7BDE82C
:10804000F08100BF253200200C32002010B54068BE
:108050000B4902798C5CFF2CE3B20DD0FE2B0DD0C6
:10806000006803F5A87350F82330064850F8220042
:10807000984203D1FF238B54002010BD0120FCE760
:1080800020320020303200202DE9F74F036890465F
:1080900093F82120022A04460F4640F098800C26CF
:1080A0004E439A195268904509D1DB691BB90020EB
:1080B00003B0BDE8F08F426810799847F7E7FFF703
:1080C000C5FF8346002840F084806368DFF8109184
:1080D0001B79FE2209F80320256895F8200002F09C
:1080E0007FFCB8F1000F1FD12E44707A02F078FCAB
:1080F000307A02F05DFC63681B79FF2209F80320E7
:108100000C2303FB07552368C5F80480DB69002BAB
:10811000CDD063681A79304B03EB42030221D95565
:10812000606802F087FBC2E7A969884507D32E443F
:108130001FFA81F8307A02F053FC707AD9E707EB26
:1081400047034FEA830A05EB830360685A6891424C
:1081500038D0904536D25B46032102F03DFB636880
:1081600095F820B0196855F80A002E4401F5A6715B
:10817000B37A01911BB301F07DFE02460199584686
:1081800002F0F6FB95F8200002F012FC63681B7900
:1081900009F8037063681A79104B43F822800C26A3
:1081A00006FB0756606800234246394602F014FB7E
:1081B000307A02F0FDFB707A02F0FAFBA0E701F0E2
:1081C00045FEDAE70379FF2209F80320E7E70820F4
:1081D0006EE711206CE700BF25320020303200200E
:1081E0002032002003681B8B5A436423B2FBF3F256
:1081F00092B2FFF749BF00002DE9F04F2DED028B41
:1082000089B0044603928A46002900F0338106684B
:1082100096F82130002B40F02F8102F0F9FB08B1D5
:10822000852846D101F044FD002839D04FF0704335
:10823000924AD3F8E83F03F0F003303B18BF012324
:108240001370FF2386F820304FF6FF73002233812E
:108250004FF0FF33F2723360F275B382F36006F1D0
:10826000200002F02DFB074600BB0AF10803804600
:1082700004935AF828205FFA88F308EE103A531C4A
:1082800000F09280256895F82110B9B108252046A4
:10829000FFF782FE284609B0BDEC028BBDE8F08FE7
:1082A00001F0CEFC0028C1D00325F3E72046FFF7FC
:1082B00073FE0425EEE74FF00108DAE7049B059210
:1082C00013F808B00C2303FB08F905EB090310466B
:1082D000596083F80AB003238DF81830BBFA8BF38A
:1082E0005B098DF8193006A901238DF81A3001F0C9
:1082F000E9FC90B9059A45F80920012393404FF015
:10830000A042BBF1000F00F0A780C2F80C3509F1C4
:108310000800284402F0D4FA08B10425B7E709F1AF
:108320000900284402F0CCFA0028F6D10C2303FB04
:1083300008530593187A02F053FB059B587A02F014
:108340004FFB55F80900BBF1000F00F0888001F0E9
:1083500091FD834655F8090001F078FD62681168C7
:108360000C2202FB08554FEA880303F5A073194459
:1083700081465A46287A02F0FBFA6368687A1968DF
:108380004A4601F5A47102F0F3FA0123EB72636827
:108390003B4A1B7902EB4303002203F8082018EE46
:1083A000101A2046FFF770FEB8F1000F83D0DAF8FC
:1083B0001030B3F5805F01D3092F58D12F4B1B78B4
:1083C00013B1012F38BF012700238DF819306068E1
:1083D0008DF818704FF4E063ADF81A300379294A2C
:1083E000079306A902F044F9054600287FF44FAF31
:1083F0006068DAF810200368D3F81075FFB24FEA0E
:10840000127CC7F1200112010CFA01F1A7F120033F
:1084100022FA07F72CFA03F30F431F434FF001082A
:10842000B76102F0D5F904233A466068CDF80080C0
:10843000022102F0EAF90221606802F00EFA039BC1
:10844000F3616368104A1B7986F8218042F8234063
:108450000E4AFF21D1541DE7C2F8083557E701F055
:10846000F5FC834655F8090001F004FD76E75B084A
:1084700001379EE70B250DE708250BE74432002066
:1084800025320020F17F02000C3200202032002033
:108490002DE9F0470768DFF86890002604463D465E
:1084A000B0464FF00C0A63681B7909EB430303F8ED
:1084B0000680EB7A73B1236828680AFB0633997A41
:1084C000B1FA81F1490901F0DDFC286801F08EFC68
:1084D000C5F804800C357EB16368084A1B79FF211A
:1084E000D154606802F074F9606802F029F902233F
:1084F00087F82130BDE8F0870126D4E7203200203C
:10850000253200202DE9F0470546D0E9007002F041
:1085100025F96868022102F0A0F997F8200002F01E
:108520005FFA3C4600264FF001094FF00C0A4FF06D
:10853000A048E37A8BB12B6820680AFB063309FA5E
:1085400000F29B7A8BB9C8F8082501F061FC207A0B
:1085500002F046FA607A02F043FA0C341EB187F852
:108560002160BDE8F0870126E3E7C8F80C25ECE7B9
:10857000826810B504462AB14369016800699847CA
:108580000023A36010BD0EB403B5039921B104AB61
:1085900001AA0193FFF758FA02B05DF804EB03B0AB
:1085A0007047000070B5064D0646002455F8043BA0
:1085B0000BB1304698470134042CF7D170BD00BF91
:1085C000543200204388033300EB830399420BD3DA
:1085D00082884FF6FF739A4208D0038833B18068CF
:1085E000431C584258417047022070470120704791
:1085F0000B4A0C495388142000FB0311CB6833B994
:108600000420496810700122074800F0FFBD0749A7
:108610000523137002238B80012209680023F3E7EE
:108620006C32002088320020D82A002050330020ED
:1086300007B5002305490093054A09680548082342
:1086400000F04AFD03B05DF804FB00BF503300208A
:10865000C8F20200D82A002007B500230146009383
:10866000034A0448082300F037FD03B05DF804FB1B
:10867000C0F20200D82A002013B500230C46009354
:108680000146084A0848042300F026FD38B9074B84
:10869000142101FB043101230B7402B010BD48F218
:1086A0000D60FAE7BCF20200D82A002088320020D0
:1086B00037B50A480A4B42689C88196853880325D5
:1086C000033305709BB2002000909B0001EB8401F6
:1086D000044800F001FD03B030BD00BF6C32002043
:1086E00050330020D82A002010B501460448FEF778
:1086F000ECFF1C220446002106F04AF9204610BD7A
:108700003C33002068B10268084B9A4209D14068A6
:10871000074B984207D00133984214BF0320012031
:108720007047032070470020704700BFDEC0ADDEF9
:10873000FE011EF12DE9F0410D460223154F2B805D
:10874000164600F5805100F108044FF001088C42F4
:108750000ED2236801330BD02046FFF733FF48B118
:108760000EB186F80080022809D14FF480632B8077
:10877000BDE8F081A3683A68934200D93B602B883A
:108780006288033313442B806388033304EB830430
:10879000DDE700BF8032002038B5144B14220D46AF
:1087A00002FB00302B68446804F58051A3B15C885B
:1087B000033403EB84048C4215D22368013312D0B6
:1087C0002046FFF7FFFE012808D002280BD0002822
:1087D000F1D12C60012038BD0834ECE76388033305
:1087E00004EB8304E7E70020F5E700BF88320020B0
:1087F000426873B504460D466AB3234BD9688A4272
:1088000029D31B699A4226D812F0030323D11F49AA
:108810000089098988421ED12068916888421AD14E
:108820001B4841688A4203D901F580518A420DD321
:1088300081698A420CD901F580518A4208D201220D
:108840002A80B3FA83F0400902B070BD1A46F7E7F8
:1088500048F20963F5E700262E800196288801A9D1
:10886000FFF79AFF30B92B8801339BB2012B2B8085
:10887000F3D9E9E7019B226899689142EED16360E0
:10888000024B1B892381DFE7D82A00206C320020AD
:10889000883200202DE9F8431C461D4B1B78064604
:1088A0000F46154673B382B37CB3DFF86C804FF08C
:1088B0001409A388012B02D948F2096020E009FBC2
:1088C00003F318F803302BB9A0882146FFF764FFA3
:1088D00020B92060A3880133A380EAE723681EB192
:1088E000998832889142EFD11FB119883A88914214
:1088F000EAD19A68C5E90023064B1B892B81002029
:10890000BDE8F88348F20160FAE748F20460F7E74F
:10891000643200206C3200208832002008B5074BFA
:108920005888191DFFF738FF18B1BDE80840FFF758
:10893000BFBEBDE80840FFF75BBE00BF6C32002041
:108940002DE9F047A24FDFF8AC8288B006463B68BD
:1089500023B9A0484146FEF7F2FE38603D68297809
:108960004B1E052B07D8DFE813F020007A007A00B1
:108970000C010C01630148F20E641422002103A8CB
:1089800006F006F841F61D539C4208BF00243B68E0
:1089900004941A78023A042A00F20282DFE812F004
:1089A000E301EF011102190220022EB18A4B0022CD
:1089B0005A604FF40644E0E72B79032B1CD8DFE81C
:1089C00003F014022A35854A1378022B1AD0137D3E
:1089D000022B4FF0010317D114214B43D118002073
:1089E000D0544868FFF738FE03E001232B71FFF7EE
:1089F0001FFE002800F0BF80774B00225A6048F22B
:108A00000D64BAE70023E7E7734A1370002353604D
:108A100041F61D54B1E772497248002302222B71BE
:108A20008A800968012200F0F1FBE2E76C4C002625
:108A30002E712068FFF710FE6B4BDFF8A0C15B883A
:108A40002568142253430CEB03020CF803605168B1
:108A50005560A588158102222160A280C9E7B5F87A
:108A600014A0AA7DDFF87491AEB1022AEB8806D972
:108A7000142101FB0A91DA1C088902440A8114229C
:108A800002FB0A99C3F57F43B9F80A20FD3313446A
:108A9000A9F80A308DE7142303FB0A9318895C6850
:108AA00004EB8004062A69D8DFE802F0274E36443A
:108AB0001D5A040041F61D54AA7DEB88022A06D9EE
:108AC000142101FB0A91DA1C088902440A8114224C
:108AD00002FB0A99C3F57F43B9F80A20FD3313441A
:108AE000A9F80A3049E74148414900234360AB698E
:108AF0000360FFF77DFE00285BD00223AB750023E7
:108B000000930423EA182146364800F0E5FA0028CD
:108B100031D048F20D64CFE72B69002B14BF03233B
:108B20000123AB750023009305F10C02042304F12B
:108B30000801E9E70123AB750022EB8800922A695E
:108B40009B0004F10C01DFE703290CBF052306237A
:108B5000AB7500230093042305F10802E118D3E765
:108B60000623AB75224B1988204B5868FFF784FD0C
:108B700004460028A0D108B0BDE8F08748F20E6492
:108B80009AE7002E7FF415AF2B79012B34D0022BFE
:108B90003FF43EAF002B7FF4EEAE02232B710DF1BC
:108BA0000A01EB68039303A8CDE90466FFF720FEF2
:108BB00010B948F20964E0E60498BDF80A10838809
:108BC000EB8003882B81FFF757FD044629E000BFA7
:108BD000843200203C3300206432002088320020A0
:108BE00050330020D82A00206C3200204832002068
:108BF0005C3300207C320020DFF8009203AA4B4651
:108C00003146A81DFFF746FE044670B9B9F80410B6
:108C10000498FFF731FD044648F209639C423FF493
:108C2000F7AE002C7FF4A9AEA5E7C9E90066F3E72B
:108C3000002E7FF4BEAE6C4B1A7BBAB11E731A784D
:108C4000013A062A3FF697AE01A151F822F000BF83
:108C5000FB8C0200218D02003F8D0200458D020039
:108C6000778902004B8D02005D8D02001A78072A79
:108C7000E5D801A151F822F0998C02003F8C020046
:108C80003F8C0200BF8C0200D38C0200F78C0200E4
:108C9000F78C0200BB8C02001A89544901321A81F8
:108CA00000225A801A730A78B2FA82F252099A7232
:108CB0000A7DB2FA82F25209DA72012207E04C49C7
:108CC00058688A884088033202448A8002221A70D7
:108CD000B5E75C88454A4649142505FB0422086827
:108CE000546850608888108102200C6088800021C0
:108CF00011740622EBE70722E9E79A7A32B9DA7AA9
:108D00008AB900221A705A805A6081E637490022D7
:108D10009A72CA68002AF2D1097C0029EFD05A80E1
:108D2000FFF7FCFD51E70022DA72304A116A002990
:108D3000E7D192F82420002AE3D00122EFE7FFF7E1
:108D4000B7FC42E7FFF754FC3FE75A88274B142152
:108D500001FB02335868FFF77FFC36E700225A60B8
:108D6000FFF766FC31E701228DF80C201A89ADF877
:108D700018209A88DB68ADF81A20059310E00222CB
:108D80008DF80C201A89ADF818209A88ADF81A20B1
:108D9000DA689B7D05929A1F534253418DF81C302F
:108DA00003A8FFF7FFFB0026414612483E60FEF78E
:108DB000F1FC11480121FEF76CFD00287FF4C7ADDE
:108DC000D9E603228DF80C20DA88ADF818201A892C
:108DD000D0E704228DF80C20DB88ADF81830DFE7EF
:108DE00005238DF80C30DBE76C3200208832002040
:108DF000503300203C3300204C33002060330020EF
:108E00004068FFF79DBD000008B505480121FEF749
:108E100028FD18B9BDE80840FFF792BD08BD00BFA6
:108E20004C33002008B5034607480268042A08D0DE
:108E30000168064A42F821300121FEF71EFD00209C
:108E400008BD48F20B60FBE7583300205432002085
:108E50002DE9F04F89B01422002103A805F098FDF8
:108E60007A4B1B7803F0FF0B3BB103A8FFF79AFB8B
:108E70000027384609B0BDE8F08F744B181DFEF787
:108E800014FD0028F4D1DBF8F83FDFF8E0A15C1C0A
:108E900008BF4FF010234FF0805208BF5B69116983
:108EA0005269581C08BF02FB01F3CAF81030684928
:108EB000A3F5405300225046CAF80C3000F0DAF80F
:108EC00007460028D5D11C2362496348DFF8A091EA
:108ED0008C22FEF7C5FB0323B8463D4601933C4672
:108EE000DAF80C6046443046FFF70CFC012862D0EB
:108EF000032817D000283DD158494FF0140C0CFB23
:108F000004FC01EB0C0201F80C0056600CF110029D
:108F10000CF1080C0A4430466144FFF70BFC45F0A5
:108F2000020545E03268531C02D04D4B9A4234D1C1
:108F3000321D06F58051106801302ED10432914265
:108F4000F9D1D9F800203AB90222C9F80060A9F88D
:108F500004204FF0010B0BE0142262433F4B022030
:108F6000991898543F4A4E60548001340881A4B245
:108F700045F0010508F58058B8F5405FB0D1019B78
:108F8000012B98BF0025EDB2022D03D0062D32D063
:108F9000002D39D148F20A676BE7019B2F495A1E11
:108FA00093B21422624388180193466003208854C8
:108FB0000134A4B2DEE7BBF1000F0DD0274B142221
:108FC0006243991802209854D9F800204A60254A33
:108FD000088154800134A4B200222349C9F80060FA
:108FE0003046FFF7A7FBB9F80420022A0CBF042281
:108FF00008221543BEE7154A0123137003A8002376
:109000005360FFF7CFFA34E702A8FFF76DFBC8B152
:109010000123013D03700A2D09D8DFE805F0060899
:109020000608070807080F110F000023037102A9A3
:109030000948FEF774FBFFF7E7FE1AE70323F5E79D
:109040000223F3E748F2076713E700BF643200200A
:10905000ACF40200B03200203C3300208832002003
:10906000DEC0ADDE6C32002054330020D82A002050
:109070005033002013B50B46114680B9104B1148F0
:10908000114AC01A0E23C0080093104B0004104967
:1090900040F00100FDF7ABFC0E2002B010BD4BB953
:1090A000074B08480B4AC01AC0080E23009300045F
:1090B000064BECE703601B6802B0BDE810401847A0
:1090C00028EB0200A8EB0200D0F202008CF40200B0
:1090D000D5F2020004F302002DE9F743DDF8288001
:1090E00088B93E4B3E483F4AC01AC0080E243E4B4A
:1090F000009400043D4940F00100FDF778FC204653
:1091000003B0BDE8F0834AB9344B3548384AC01A39
:10911000C0080E24344B00940004EBE7D0F800E0C4
:10912000BEF1000F09D12D4B2D48324AC01AC0089C
:1091300008242D4B00940004DCE74BB9274B28484A
:109140002D4AC01AC0080924274B00940004D1E717
:109150004568D5F80490B3FBF9F509FB15354DB119
:109160001E4B1F48254AC01AC00809241E4B0094F4
:109170000004BFE78D0709D0184B1948204AC01AD0
:10918000C0081024184B00940004B3E712F0030F3A
:1091900009D0124B12481B4AC01AC0081024124BA7
:1091A00000940004A6E7C568A9420DD34D1EEC1833
:1091B0000569AC4208D8CDF82880DEF80C40A446FA
:1091C00003B0BDE8F0436047044B05480E4AC01A9F
:1091D000C0081024044B009400048BE728EB020025
:1091E000A8EB0200D0F2020079F40200D5F20200EE
:1091F00052F30200FEF2020011F3020058F30200E3
:1092000082F302009AF30200BDF30200F7B580B9C1
:109210002A4B2B482B4AC01AC0080E242A4B009414
:1092200000042A4940F00100FDF7E1FB204603B0AD
:10923000F0BDD0F800C0BCF1000F09D11F4B204891
:10924000234AC01AC00808241F4B00940004E8E712
:109250004AB91A4B1A481F4AC01AC00809241A4BA7
:1092600000940004DDE74568D5F800E00EF1FF3515
:109270000D4209D0114B1248174AC01AC0081024D9
:10928000114B00940004CCE7C568A9420CD34D1ED5
:109290000EFB02540569AC4206D8DCF81040A44627
:1092A00003B0BDE8F0406047044B05480B4AC01AC4
:1092B000C0081024044B00940004B2E728EB02001D
:1092C000A8EB0200D0F2020066F40200D5F2020020
:1092D000FEF2020011F30200E4F302000AF40200BD
:1092E00029DF704728DF704770B503689E6886B035
:1092F00004460D466EB114220021684605F048FB75
:10930000A3680593237901952BB1012B0DD06846F5
:10931000B04706B070BD01238DF800302369029379
:10932000E368039363690493F1E702238DF8003047
:10933000E3681B030293F5E7084670470020704777
:10934000024B187A003818BF0120704704340020FF
:10935000034B187A0122B0FA80F05A744009704722
:109360000434002008B510461A4605F0E8FA00203B
:1093700008BD000008B514220021044805F008FBD0
:109380000348FEF780F9002008BD00BF0434002028
:10939000F433002010B5094C094B43602046FEF71A
:1093A00084FA40B904F06EFE064920741C23064876
:1093B0008C22FEF755F9002010BD00BF04340020B8
:1093C000A0F4020068330020F433002038B5234DA8
:1093D000234C2B7A3BB923492348FEF7B0F9206090
:1093E00008B9686038BD022324682B72237973B1F1
:1093F000012B24D020460321FFF776FF00232B7298
:109400006B6018491848BDE83840FEF7C3B9D4E985
:109410000523D21AB2F5805FD4E9031028BF4FF4B8
:1094200080529208012A38BF012219441844FFF7DC
:1094300057FF50B11128DDD101232B72D2E7D4E9B7
:1094400003031844FFF74EFFF3E72B7C002BC9D131
:10945000BDE83840022000F009B800BF0434002005
:109460001C34002018340020F433002038B5234C7D
:10947000237A002B41D0022B09D1032830D0204B76
:1094800000221B68E2601A793AB1012A22D0637C7B
:109490007BBBBDE83840FFF799BFD3E905128D1AB1
:1094A000B5F5805F94BF521902F580529A619142DE
:1094B000EDD102284FF0000308BF19462372104B6C
:1094C00018BF0D211868FFF70FFF0E490E48FEF771
:1094D00061F9DCE71A6901321A615B699A42E7E7D0
:1094E000E3680133082B01D8E360D0E70023E36091
:1094F000DFE7BDE8384004F0B5BD38BD04340020D6
:109500001C34002018340020F4330020831E012B6B
:1095100001D8FFF7ABBF704700F0FD03012B08D166
:10952000044B00225A74421E504250411874FFF7F7
:109530004DBF70470434002010B5064C201DFEF7C7
:10954000B4F928B9637C1BB9BDE81040FFF73EBFF2
:1095500010BD00BF043400202DE9F34180460D46C4
:10956000104801A916461F46FEF7AFF80446B0B1F1
:1095700018220021043005F00BFA2D0B0123237172
:1095800001A90848C4F80080A760E5606661FEF79D
:10959000C6F8FFF7D1FF002002B0BDE8F08104203B
:1095A000FAE700BFF43300202DE9F34180460F466F
:1095B0000F4801A916461D46FEF787F80446A8B1D4
:1095C00018220021043005F0E3F9089BA36001A9EB
:1095D000C4E903670648C4F800806561FEF79FF898
:1095E000FFF7AAFF002002B0BDE8F0810420FAE7EF
:1095F000F43300204FF08053D3F83001421C04BFF5
:109600004FF0704393F8E00F831F58425841704762
:109610004FF0704393F8E02F062A09D1D3F8E83FC2
:10962000C3F30313033B032B02D8024AD05C7047F9
:1096300000207047D4F4020008B5FFF7DBFF40B10B
:109640004FF080538F4AD3F82433C3F30423C2F876
:109650004035FFF7DDFF10B18B4B8C4A5A67FFF79F
:10966000C9FF48B14FF080534FF08042D3F84432E5
:10967000C3F34233C2F83C35FFF7CAFF30B1844A26
:10968000D2F8FC3023F08073C2F8FC30FFF7B2FF51
:1096900040B14FF080430022C3F80C21C3F81021E1
:1096A000C3F83825FFF7B4FF20B14FF08043032201
:1096B000C3F8A025FFF7ACFF60B1764B0522C3F8D5
:1096C00010260122C3F888260022C3F818263F225C
:1096D000C3F814264FF08053D3F83021511C09BF32
:1096E0004FF07043D3F8343193F8E02FD3F8E83FCC
:1096F00008BFC3F30313062A4DD1033B032B03D842
:10970000654AD35C002B46D04FF08052634BD2F8B1
:109710000414C3F82015D2F80814C3F82415D2F89D
:109720000C14C3F82815D2F81014C3F82C15D2F86D
:109730001414C3F83015D2F81814C3F83415D2F83D
:109740001C14C3F84015D2F82014C3F84415D2F8FD
:109750002414C3F84815D2F82814C3F84C15D2F8CD
:109760002C14C3F85015D2F83014C3F85415D2F89D
:109770003414C3F86015D2F83814C3F86415D2F85D
:109780003C14C3F86815D2F84014C3F86C15D2F82D
:109790004424C3F87025FFF72DFF48B14FF08053E4
:1097A0004FF08042D3F8583203F04F03C2F8E43E42
:1097B000FFF720FF48B14FF08043D3F80024D207D1
:1097C00044BF6FF00102C3F800244FF08053D3F878
:1097D0003021062A0ED1D3F83431033B032B02D8B3
:1097E0002F4AD35C33B12F4AD2F83C3743F480631D
:1097F000C2F83C37264AD2F8883043F47003C2F8E6
:109800008830BFF34F8FBFF36F8F4FF01023D3F823
:109810000022002A03DBD3F80432002B2EDA224B7D
:109820000122C3F80425D3F80024002AFBD04FF00E
:1098300010221521C2F80012D3F80024002AFBD010
:109840004FF010231522C3F80422174BD3F800243D
:10985000002AFBD00022C3F80425D3F80024002AF4
:10986000FBD0BFF34F8F0A49104BCA6802F4E06285
:109870001343CB60BFF34F8F00BFFDE70C4B0D4A86
:109880001A6008BD0030014000C007400DF0ADBABD
:1098900000ED00E000500040CCF4020000C00040A9
:1098A000D0F402000010004000E001400400FA057E
:1098B000FC2A00200090D003054A4FF0A043105C22
:1098C000D3F8043523FA00F000F00100704700BF20
:1098D000DAF40200044B1A5C012393404FF0A042DB
:1098E000C2F80835704700BFDAF40200044B1A5C76
:1098F000012393404FF0A042C2F80C35704700BFDF
:10990000DAF4020008B50020FFF7F0FF0120FFF7AE
:10991000EDFF0220FFF7EAFFBDE808400320FFF754
:10992000E5BF08B50020FFF7D5FF0120FFF7D2FF04
:109930000220FFF7CFFFBDE808400320FFF7CABFB2
:10994000074A4FF0A041105CD1F804350122824053
:1099500022EA03001340C1F80805C1F80C3570472E
:10996000DAF40200054A4FF0A043105CD3F810353A
:1099700023FA00F0C04300F001007047D8F4020061
:109980000D2805D00E280CBF01204FF0FF30704786
:1099900000207047C20708B501460CD54FF0A04320
:1099A0000322C3F84427C3F84827C3F84C27C3F859
:1099B0005027FFF7A7FF8B0741BF4FF0A0430C22B2
:1099C000C3F83427C3F8382708BD000038B5074C62
:1099D000051E04F1080318BF1C4623682BB11A6842
:1099E00022605B6828469847F7E738BD2834002096
:1099F00020B9054B01225A70FFF7E8BF012802D1B8
:109A0000014A9070F8E770472034002020B9034BDA
:109A100001225A70FFF7DABF704700BF20340020E0
:109A200038B50E4C2378B3B90D486360A360236149
:109A3000E36000F075F8054604F024FB08B900F077
:109A40007BF801232370074BD3F800340BB10123BB
:109A5000A370284638BD8525F5E700BF20340020D7
:109A6000F19902000000014037B50D4C00230DF1C3
:109A700007008DF80730FDF77BFCE368013BE360EE
:109A8000E36833B9074BD3F8005415B900F066F812
:109A9000A5709DF80700FDF78FFC03B030BD00BF37
:109AA0002034002000000140012813B50CD0032809
:109AB00020D038B9134B0122C3F88020BFF34F8F59
:109AC000BFF36F8F02B010BD0F4C00230DF10700E4
:109AD0008DF80730FDF74CFC23780BB9FFF7A0FF9A
:109AE000E3689DF807000133E3600123A370FDF7ED
:109AF00063FCE7E700F020F802B0BDE81040FFF794
:109B0000B3BF00BF00E100E02034002000F180403E
:109B1000002382B0036003680193019B02B0704789
:109B2000044A137923B901211060918018467047C7
:109B30008520704734340020074B1A68D20704D4BC
:109B4000C02283F8002301221A604FF080430122D3
:109B5000C3F81825704700BF00E100E04FF08042D5
:109B600008B50223C2F808334FF48270FFF7CEFF26
:109B70000123D360D2F81834DB03FBD408BD000006
:109B80004FF0804110B5D1F8003163B14FF48070CF
:109B9000FFF7BCFF0D4B58790122C1F8082310B91B
:109BA0005A711B6898474FF08042D2F8043163B174
:109BB0004FF48270FFF7AAFF0223C2F80833034B69
:109BC000BDE810401B680120184710BD3434002048
:109BD00000F1804000F5C040002382B003600368BC
:109BE0000193019B02B07047800000F1A040D0F8C3
:109BF000002722F44032C0F80027D0F8003743EAAB
:109C00000141C0F800177047054B4FF0FF3207289D
:109C100043F8202084BFC01880F84820704700BF58
:109C20003C340020C208054900F0070001238340AE
:109C3000885C20EA03008854704700BF90340020FD
:109C400010B5184991F8583053BB4FF0FF3222FA43
:109C500003F0C00748BFC81803F1010348BF80F8EC
:109C60003020202BF3D10024E0B20134FFF7CCFFE9
:109C70000C2CF9D10C4B0022C0204A6583F8060356
:109C8000402018604FF4BE70FFF7A2FF074B4FF063
:109C90000040C3F80403012381F85830104610BD7A
:109CA0000820FCE73C34002000E100E000600040B8
:109CB000034B93F85800003818BF0120704700BFCD
:109CC0003C34002030B52E4B1A1892F93040013444
:109CD00053D18C78002C4CD01C46002254F8045BE5
:109CE000013541D11C1884F83020002443F822406B
:109CF000920002F1804202F5C0420B78D2F8105572
:109D00004C7825F498151B04240525F4F85504F423
:109D1000801403F44033C2F8105523430402D2F8F0
:109D2000105504F4F85423432B43C2F810354A78F5
:109D30000123012A4FF0A04203FA00F30CBFC2F83E
:109D40000835C2F80C3500F5E073032142F8231002
:109D5000C2080C49012300F0070003FA00F08B5CF5
:109D600018438854002003E00132082AB6D10420A9
:109D700030BDFE2382F83030D9E70820F8E700BF75
:109D80003C3400209034002038B5164C251801468C
:109D900095F83000072809D8FFF736FF95F93030DD
:109DA000114A03F5A273002042F823006318FF2232
:109DB00004EBD10483F8302094F8542001F007001C
:109DC000012383401A420BD04FF0A04301F5E0720B
:109DD000022043F82200BDE838400846FFF722BFC2
:109DE00038BD00BF3C34002000600040074B1844E1
:109DF00090F930309B0003F1804303F5C043D3F862
:109E0000102542F00302C3F8102570473C340020AF
:109E1000074B184490F930309B0003F1804303F561
:109E2000C043D3F8102522F00302C3F81025704771
:109E30003C340020044B184490F930000C30800072
:109E400000F0FC00704700BF3C34002008B5FFF76D
:109E5000F1FF00F1804000F5C04008BD044B1844FC
:109E600090F930001830800000F0FC00704700BF0F
:109E70003C34002008B5FFF7F1FF00F1804000F509
:109E8000C04008BD0A4B1844003990F930304FEA01
:109E9000830303F1804303F5C04318BF0121D3F8C6
:109EA000102522F4801242EA0152C3F810257047AF
:109EB0003C340020F0B5394E331893F93030002B84
:109EC00069DA8D78C5F34005002D0BBF0823002308
:109ED0000C240824A34201D10420F0BD56F82370BD
:109EE000013743D137185CB246F8232087F8304059
:109EF00015B9F21882F848008A78550716D4D707A2
:109F000036D5820002F1A042D2F8005725F00205B2
:109F1000C2F80057224FC50800F0070C012202FAD0
:109F20000CF217F805C042EA0C027A558A780D78CF
:109F300012F0020225D09B0003F1804303F5C043D9
:109F40000002D3F8102522F4473222F44072C3F8FD
:109F500010252D04D3F8102500F4F85005F44035F1
:109F600028431043C3F810050020B6E70133B1E7DA
:109F70004D7800F5E0724FF0A047AD0047F8225051
:109F8000C8E7083C46FA84F494F8500040EA851586
:109F900084F85050E8E708209FE700BF3C340020D9
:109FA0009034002038B5204C251895F93020072A28
:109FB00018DD083A44FA82F494F850309B09032BD8
:109FC0000BD14FF0A043D3F81015C14001F00101AF
:109FD0000231BDE83840FFF707BE012B0CBF02215C
:109FE0000321F6E7D3B2072B1DD8930003F180437A
:109FF00003F5C043D3F8100540F00100C3F8100585
:10A0000002F1400040B2800080B2FFF7E1FD51B1A3
:10A0100095F9303054F823302BB1012303FA02F2C2
:10A02000024BC3F8042338BD3C34002000600040DC
:10A030004FF0A043D3F8103523FA00F000F00100F0
:10A04000704700002DE9F74F00244E4D01944FF466
:10A050008072012102F1804303F5C04390B21B6876
:10A06000012B06D1D5F804330B4202D0FFF7B0FD27
:10A070000C430432B2F5907F4FEA4101EAD1414BE3
:10A08000D3F87C31012B0CD14FF4BE70FFF7A0FD4B
:10A090004FF0A04344F00044D3F820250192C3F8C8
:10A0A0002025E3B2D3B1384F00250126344210D029
:10A0B000AB0003F1804303F5C043D3F81005D3F898
:10A0C000101557F8253023B1C1F30141C0F3042026
:10A0D00098470135082D4FEA4606E7D1002C48DAAB
:10A0E000294D4FF0A048294E4FF00009012716F9DD
:10A0F000013B5A1C31D0C3F3C20202A90A44DCB2AC
:10A1000012F8042C03F03F0A03F0070307FA03F3E5
:10A110001A4222D00AF5E073504658F82330C3F3B0
:10A12000014BBBF1020F0CBF03210221FFF75CFDC5
:10A1300007FA0AF3C8F8203505EB0A0393F9303023
:10A1400055F823304BB1A109032904D0BBF1020F0C
:10A1500012D1012901D15046984709F10109B9F1FD
:10A16000040FC4D1D8F820350193C8F82035002B4E
:10A17000B9D103B0BDE8F08FBBF1030FEDD10229D7
:10A18000E8E700BF006000403C3400208C34002031
:10A19000014B1B68184700BF983400200023435030
:10A1A00082B043580193019B02B070472DE9F04102
:10A1B000224E234FDFF88C8000254FF48034D7F8EF
:10A1C000043306F5A041234289B20CD0336853B161
:10A1D000C7F848433846C7F80843FFF7DFFFD8F809
:10A1E0000030E8B298470135032D4FEA440406F1E8
:10A1F0000406E4D11248D0F80433DA070AD5D0F8BF
:10A2000000313BB14FF48071FFF7C8FF0D4B0420C4
:10A210001B6898470A48D0F804339B070CD5D0F840
:10A2200004314BB14FF48271FFF7B8FF054BBDE825
:10A23000F0411B6805201847BDE8F08140B100409F
:10A2400000B00040A034002000F1804000F5E04064
:10A25000002382B0036003680193019B02B0704742
:10A26000F0B5524B524CD3F8043185B0002B3DD0A1
:10A2700094F82E204FF48270FFF7E6FF2AB394F88B
:10A280002F3013BB494AD2F80031002B32D04FF4A3
:10A290008070FFF7D9FF638B94F82D00834250D96B
:10A2A00021891B1A9BB289B26383CB1A616801EBC7
:10A2B0004303C2F82C36C2F830064FF48270FFF721
:10A2C000C3FF3A4B01225A6014E06368029323896A
:10A2D000ADF80C30E36800218DF8041033BB237413
:10A2E000236801A89847002384F82F3094F82E3073
:10A2F000002BC7D12D4BD3F810315BB14FF48870D0
:10A30000FFF7A2FF0023237402238DF8043001A875
:10A3100023689847254BD3F81431EBB14FF48A707A
:10A32000FFF792FF0023237405B0F0BD208B6083FC
:10A3300063602081E160002AD2D11C4B01221A60A7
:10A34000CEE7BAD1E368012184F82F1013B10021C0
:10A350006183AEE76383B0E766694FF0004701258C
:10A36000002EE1D0B6FA86F227FA02F346329200C6
:10A3700026EA030602F1804303F5E0431B68002B45
:10A38000EED01046A2F58C72FFF75EFFD30882F084
:10A390000402C2F380028DF808308DF8045023685F
:10A3A0008DF8092001A89847DAE700BF0070004047
:10A3B000A434002038B5204A92F82C300446002BF3
:10A3C00037D111601D490078C1F8F0056078C1F8F7
:10A3D000F4050125E078137482F82D30536182F87A
:10A3E0002F306FF0004382F82E0082F82C504FF48B
:10A3F0008270C1F80833FFF727FF4FF48070FFF732
:10A4000023FF4FF48A70FFF71FFFA3780C485B010E
:10A41000DBB280F80733802303600223C1F80433E2
:10A4200092F82E300BB1C1F80453C1F8005500204A
:10A4300038BD0820FCE700BFA434002000700040B5
:10A4400000E100E070B52A4B1A7C02F0FF05002AFB
:10A450004BD10A79012A9CBF264CC4F8005500F163
:10A460000C0503EB4504247924B993F82D400134FD
:10A4700083F82D4003EB4503CC790D7A8E781C715F
:10A480005D714B7836021B0106F4E06603F0300381
:10A4900033430E7806F003063343CE78360306F4D2
:10A4A00080563343160406F4E02633434E79897907
:10A4B000360506F480160906334301F080710B431C
:10A4C0000C4901EB0016000100F1804000F5E0406E
:10A4D000012AC6F81835C0F81455C0F8104502D83E
:10A4E0000123C1F80035002000E0112070BD00BF3D
:10A4F000A43400200070004070B5324A147C04F08F
:10A50000FF03002C5CD1304C012503261574C4F8E0
:10A510000863C4F82C16C4F8305692F82D40AC42AB
:10A520000CD91D46190101F1804101F5E0410133CB
:10A53000082BC1F81455C1F81055F3D100F10C03E4
:10A54000000102EB430300F1804000F5E04019797F
:10A550005B79C0F81435C0F810151B4901230B6056
:10A560004B6042F21073D1F8040108B9013BFAD1F3
:10A570004FF48070FFF768FE4FF48270FFF764FEBF
:10A58000012C11D90F4800210B0103F1804303F581
:10A59000E0430131047F457FC3F814550829C3F80F
:10A5A000104500F10200EFD192F82E10064B29B1B0
:10A5B00003210020C3F80413107470BD0221F8E7D2
:10A5C0001120FAE7A43400200070004070B5264A3C
:10A5D000264B05461220C2F808031C7C022C03D12E
:10A5E000C2F80403112070BD187C01281CD1D86862
:10A5F00018B10223C2F80433F4E7DD60198393F83D
:10A600002E305BB9D2F80031002BFBD04FF48070B4
:10A61000FFF71AFEC2F82C56C2F83016124B02226F
:10A62000C3F804230020DEE7022093F82E40C2F88E
:10A630000403012600201E745D601981D8603CB1BE
:10A64000598393F82D30C2F82C56C2F83036CAE739
:10A65000C2F82C564FF48070C2F83016FFF7F4FDA4
:10A6600016602046BFE700BF00700040A434002001
:10A67000F7B506792F4D0C237343EF183C7A002C65
:10A6800055D1EA504B687B60477903682246A4465F
:10A69000D4B2A7423CD8CA7843F307345201002C05
:10A6A000C3F30733D2B23DDB234F07EB040C8CF826
:10A6B00000230122640903F01F0302FA03F347F8A1
:10A6C000243003684A78D3F8040502F0030220F02E
:10A6D00003000243C3F80425D3F808058A7820F064
:10A6E000030002F003020243C3F80825D3F8100563
:10A6F0000A7820F00F0102F00F020A43C3F8102578
:10A700000C2303FB065501232B72002003B0F0BD80
:10A71000940004F5A074013243F804C01C5901945C
:10A72000019CB5E7054C03F00F03E254C9E708208C
:10A73000ECE700BFD434002000E100E014ED00E0BD
:10A74000036801221A600279034B0C2101FB0233DA
:10A7500002221A72704700BFD4340020036801221D
:10A760001A610179024B0C2000FB01331A72704709
:10A77000D434002038B503681A0B43F30733002B99
:10A7800004460CDB02F01F015B0901228A402033E2
:10A790000D4941F82320BFF34F8FBFF36F8F23681C
:10A7A0000025D3F80022C3F800524FF0FF32C3F85F
:10A7B00008232046FFF7D2FF2279044B0C2101FB2E
:10A7C00002331D7238BD00BF00E100E0D434002028
:10A7D00003680122DA60704737B54FF480340068AF
:10A7E0008C407BB18B0003F5A0730025C550C35886
:10A7F0000193019BC0F8044301F5A87140F82120A2
:10A8000003B030BDC0F80843F6E770B4046840F206
:10A810000116D4F800528E4025EA0605C4F800520D
:10A82000D4F800522B43C4F800329DF80C3070BCB1
:10A83000FFF7D2BF8B0003F5A07302689BB2002024
:10A84000D05082B0D3580193019B4FF4803303FA68
:10A8500001F1C2F8041302B0704702684FF480336C
:10A8600003FA01F1C2F80813704700002DE9F34123
:10A87000104C114F114E00254FF48038236883B1DE
:10A88000D7F8043308FA05F21A420AD000232360ED
:10A890002368019304F5E040019B80B2D6E90031C2
:10A8A00098470135042D04F10404E7D102B0BDE856
:10A8B000F08100BF4091004000900040D43400205F
:10A8C0002DE9F74F4FF00009154D164F06464FF092
:10A8D000040AC8465FFA89FB01240DF1070004FA57
:10A8E0000BF48DF80780FCF743FD2C4208D03B6841
:10A8F00014EA030201BF23433B6086F800B092468E
:10A900009DF80700FCF758FDBAF1000F03D0A543EE
:10A9100009F10109DED1504603B0BDE8F08F00BF58
:10A92000FFFF0100E0340020012337B503FA00F5F2
:10A93000C5F31003ABB10C4B0024C3F808550DF15F
:10A9400007008DF80740FCF713FD084B186820EA54
:10A95000050018609DF80700FCF72EFD204603B0A7
:10A9600030BD0720FBE700BF00F00140E0340020CD
:10A9700010B5A1B19AB101238340C3F3100484B18F
:10A980000A4C246823420ED0C00000F1804000F53C
:10A99000F830C0F81015C0F81425002010BD0E20A6
:10A9A000FCE70720FAE70820F8E700BFE0340020C2
:10A9B000012202FA00F3580C400440B91BB1064AC8
:10A9C0001268134205D0054AC2F8043570470720C3
:10A9D00070470820704700BFE034002000F00140BD
:10A9E000012202FA00F3580C400440B91BB1064A98
:10A9F0001268134205D0054AC2F80835704707208F
:10AA000070470820704700BFE034002000F001408C
:10AA1000034B187810B901221A70704785207047CF
:10AA2000E434002013B5084CD4F800314BB1074B87
:10AA30001B6898470023C4F80031D4F80031019313
:10AA4000019B02B010BD00BF00000140E8340020AF
:10AA500070B5114B1960114B1C780546D4B9104ED6
:10AA600001221A700378C6F80C3541684FF47A72E7
:10AA70000023C803490C03F09DFEC6F804052B7A99
:10AA8000084A5B01DBB282F810334FF48033136065
:10AA9000204670BD0820FCE7E8340020E6340020A2
:10AAA0000000014000E100E0044B0122C3F8042350
:10AAB0001A60034B02221A70704700BF0000014069
:10AAC000E634002037B5054600240DF107008DF867
:10AAD0000740FCF74DFC0C4B1A78072A11D8511C83
:10AAE00019700A492A70D1F80805012393400343DD
:10AAF000C1F808359DF80700FCF75EFC204603B05E
:10AB000030BD0424F6E700BFE5340020000001401A
:10AB1000034B044A00F5C07043F82020704700BF83
:10AB2000000001403546526E0220FEF709BF0000CA
:10AB30002DE9F04780460D46FEF722FF0128044626
:10AB400010D8012D10D0022D30D05DB91A48FCF775
:10AB50003AFB1A4B04EB440213449D78184B1B5DDF
:10AB6000AB4219D0BDE8F087144E00EB4003F21859
:10AB7000F55C5378470053B1DFF84C900E484A46D5
:10AB80004FF48041FCF707FB08B989F8008027449F
:10AB90003E440B4BB2781A55002DE3D0094B1B688D
:10ABA000002BDFD02846BDE8F047184700EB4004F3
:10ABB000024804446578EFE7103500205035002046
:10ABC0006535002060350020EC340020007802213B
:10ABD000FFF7AEBF08B5094B1B7853B10020FEF755
:10ABE00085FE0120FEF782FEBDE808400320FEF747
:10ABF0007DBEBDE80840FEF785BE00BFED340020F5
:10AC0000F8B57A4C237805461BB100232370FFF773
:10AC1000E1FF172D00F28780DFE805F00C171742DF
:10AC20005364757F878C878C949999999999C3C837
:10AC3000D0D8E3E3FFF7CEFF6D48FCF7C4FA6D4BC5
:10AC4000002204461A702046F8BD0020FEF734FEAC
:10AC5000F0B10020FEF74AFE022D0CBF4FF4E16474
:10AC60004FF47A64634B1D7000254FF400464FF497
:10AC70007A7029464FF4FA620023E4FB060103F0E0
:10AC800099FD2A460146BDE8F8405948FCF783BAC9
:10AC9000FEF720FE022D0CBFC8244FF4C874E1E774
:10ACA0000020FEF709FE40B10020FEF71FFE4FF422
:10ACB0004874504B03221A70D6E7FEF70BFEC824E7
:10ACC000F7E70020FEF7F8FD38B10020FEF70EFE92
:10ACD0004FF47A64474B0422EDE7FEF7FBFD4FF497
:10ACE000C874F7E70020FEF7E7FD48B10020FEF743
:10ACF000FDFD404B05221A7040F6CD410022C2E70F
:10AD0000FEF7E8FDF5E70020FEF71AFE394B0622B4
:10AD10001A70002240F26661B5E70020FEF7DAFD06
:10AD2000344B07221A7000248DE701202070FEF7B3
:10AD300007FEEEE701202070FEF702FE00224FF42E
:10AD40000051A0E7FEF7EDFD2A4B0C22EAE72A4866
:10AD50002A4EFCF738FAD5F1110504461CD0D8B9B3
:10AD6000012D13D0C820454321464FF400474FF42E
:10AD70007A704FF4FA620023C5FB070103F01AFD55
:10AD8000224601461C48FCF706FA04460220FEF75C
:10AD9000A1FD0123337056E70220FEF7A7FD002333
:10ADA000F8E7FFF717FF134B1222BBE7FFF712FF7D
:10ADB0000020FEF78FFD0F4B1322B3E7FFF70AFFCA
:10ADC0000120FEF787FD0B4B1422ABE7FFF702FFD4
:10ADD0000020FEF77FFD0120FEF77CFD054B1522CC
:10ADE000A0E7FEF79EFD034B1D709CE75C3500203D
:10ADF0003035002064350020F0340020ED34002090
:10AE0000044B1B68DB0703D5034B1878FFF7F8BE2C
:10AE1000704700BF5835002064350020012801D854
:10AE2000FEF7A0BD00207047044B1B6813F0010320
:10AE300001D0FFF7E5BE1846704700BF5835002027
:10AE400038B51A4B18601A4B10F002040546196009
:10AE500016D0184B18480F221A701022DA700221EF
:10AE600040F23332FCF72EF8044648B9FCF782F87A
:10AE7000044628B90146114A1148FCF781F90446F5
:10AE8000EB0711D50120FEF785FD6CB921460D4A6F
:10AE90000D48FCF775F9044630B9BDE838400B4A57
:10AEA0000B480121FCF76CB9204638BD583500200D
:10AEB000603500205035002018F50200CDAB0200AF
:10AEC0002CF5020001AE020030F5020029AB0200B1
:10AED00028F502000388102B02D0112B05D07047F3
:10AEE000044A1368013313607047024A1368013B38
:10AEF000F9E700BF6835002010B50C4629B10120E4
:10AF0000FFF78CFF18B102232370002010BDFFF75C
:10AF100085FF08B10B23F7E72070F6E7BFF34F8FEB
:10AF20000549064BCA6802F4E0621343CB60BFF3E5
:10AF30004F8F00BFFDE700BF00ED00E00400FA0501
:10AF40006CDF70476DDF704776DF70477ADF7047E0
:10AF50007CDF70477FDF70478FDF7047B1DF70475E
:10AF60003FDF704741DF7047014B01221A70704785
:10AF70002C3E0020F8B5037805461BB94068052132
:10AF8000FFF724FB094C0A480A4F241AE40824045A
:10AF900044F0030402266B6839469A5F2046023665
:10AFA000FBF712FD0A2EF6D1F8BD00BF78EB0200C8
:10AFB00028EB020034F502000448054B0549C01A8D
:10AFC000C008000440F00300FBF7FABC78EB020075
:10AFD00028EB02003FF50200FBF7E2BF08B5164878
:10AFE000FCF7F1F800224FF4CD711448FCF7D3F8C8
:10AFF000002210211248FCF7CEF812490320FFF777
:10B000001FFF1148032102F00FF808B1FBF7C8FF3A
:10B010000E4B0F480F4905221A700F4BC01AC0087B
:10B02000000440F00300FBF7CBFC0C4B01221A7725
:10B0300000225A6108BD00BF303E0020A03D002024
:10B04000C83D0020A1B5020048390020503E002034
:10B0500078EB020064F5020028EB0200B03E00200D
:10B0600001F078B937B51F4B1F4C0546E41A2A7812
:10B070001E4B406853F82220E408240444F00304E3
:10B0800080B91B492046FBF79FFC2B78012B13D07E
:10B09000032B11D023B96B6813B9164B01221A7018
:10B0A00003B030BD019201F003F8019A1249034642
:10B0B0002046FBF792FCE8E76B68002BF0D1AA680A
:10B0C0000E492046FBF780FCAA890D492046FBF774
:10B0D0007BFCEA890B49204603B0BDE83040FBF712
:10B0E00073BC00BF28EB020078EB020048FA0200B4
:10B0F00073F50200873D002094F50200ACF50200D4
:10B10000BEF50200CEF5020010B50446C8B1032812
:10B1100032D11A4B1A481B49C01AC008000440F02B
:10B120000300FBF74DFC184B002202209A60FFF74A
:10B130007BFE164BC8221A60F0B1BDE81040FBF749
:10B140002FBF0E480E4B12491B1ADB081B0443F09D
:10B150000300FBF735FC2046FFF766FE08B1FBF75E
:10B160001FFF0C48FDF7CEF90B48FCF72CF80B48F5
:10B17000FCF729F8FFF7D2FE10BD00BF28EB020054
:10B1800078EB0200E1F50200503E0020703500200F
:10B19000F2F502002CFA0200A03D0020C83D00207C
:10B1A0000388212B13B5044653D01AD8132B5ED035
:10B1B00013D8102B2DD0112B11D1384B38483949C9
:10B1C000C01AC008000440F00300FBF7F9FB364B3F
:10B1D0004FF6FF721A80FFF7A1FE1D2B0CD002B0B4
:10B1E00010BD522B51D0562B01D03B2BF7D1A0884C
:10B1F0001321FFF7A9FE41E0284B29482B49C01A2B
:10B20000C008000440F0030002B0BDE81040FBF7A6
:10B21000D7BB224B22482649C01AC008000440F080
:10B220000300FBF7CDFB0720FFF7FEFD08B1FBF79E
:10B23000B7FE1D4BA1881F48198002F099FC08B188
:10B24000FBF7AEFE1C4B01225A751C4B00225A61C3
:10B25000C5E7002380888DF8043001A98DF80530FA
:10B26000FFF77AFE0028BAD0FBF79AFEB7E70E4840
:10B27000002300881A468521FFF76CFE0028AED017
:10B2800002B0BDE81040FBF78BBE074800231A460A
:10B2900019460088FFF762FEF0E700BF28EB0200C6
:10B2A00078EB02004AF602000E2B002003F60200A3
:10B2B0001BF602000C3E0020503E0020B03E002055
:10B2C000F0B5037889B00546032B42D8DFE803F0D8
:10B2D000024B585F314B324C3249334FE41AE40889
:10B2E000240444F005042046FBF76AFB0026AB8AE1
:10B2F000B34230D82D492046FBF762FB2B696946E3
:10B300005A1E08460F3312F8015F01F8015B9A429A
:10B31000F9D104A900F0DAFE2549234F2046FBF7B6
:10B320004FFB04AD002615F8012B394620460136A7
:10B33000FBF74AFB102EF6D11C492046FBF740FBD9
:10B340001C4B9DF8132083F85C209DF8142083F893
:10B350005D2009B0F0BD2B6939469A5D2046FBF7A8
:10B3600033FB0136C3E70E480C4B1349C01AC00823
:10B37000000440F0050009B0BDE8F040FBF720BB39
:10B380000748064B0D49C01AC0080004F1E70448FD
:10B39000024B0B49C01AC0080004EAE728EB020080
:10B3A00078EB02007CF602009AF602004CF90200EB
:10B3B000A3F60200503E0020C1F60200DEF60200B5
:10B3C00001F7020008B503784BB9054B3B211888FB
:10B3D000FFF7BAFD18B1BDE80840FBF7E1BD08BDB5
:10B3E0000E2B002038B5054D052445F001054FF41E
:10B3F0007A40A847013CFAD138BD00BF40FA0200AC
:10B400000D4B4A881B889A4214D10A8840F677234C
:10B410009A420FD18B88094A09480A49033B9BB2DB
:10B420001380094A801AC00800041A4640F003003D
:10B43000FBF7D3BA704700BF0E2B00200C2B002067
:10B4400078EB020024F7020028EB0200FBF7A8BD0E
:10B450001FB5094A10685168127A01AB03C3074946
:10B4600007481A70FEF7A6FF01A90220FEF7EAFFBF
:10B4700005B05DF804FB00BF00FA020075AF0200E2
:10B4800034FA020008B50849084802F051FA08B138
:10B49000FBF786FD0548F72102F05EFA18B1BDE81A
:10B4A0000840FBF77DBD08BD01B40200883D0020C7
:10B4B00008B50548032101F0B7FD08B1FBF770FDA1
:10B4C000024B01221A7008BD483900207435002053
:10B4D00037B52D4CFFF786FF21460320FFF70CF808
:10B4E000FFF780FFA11C0320FFF706F8FFF77AFFA4
:10B4F000211D0320FFF700F8B4F90230B4F9000071
:10B500001844B4F9043018440323B0FBF3F007EEF9
:10B51000900AF8EEE77A17EE900A03F031F916A3D5
:10B52000D3E9002303F056F8184B002204460D46D9
:10B5300003F04CF812A3D3E9002303F04BF803F017
:10B540000BF9C3B2124A642B88BF64239374937CB3
:10B5500001932946204603F0D9F80E4C019B0E4971
:10B5600002460E48241AE408240444F0030003B001
:10B57000BDE83040FBF731BA0E2DB29DEFA7E63F94
:10B58000D9899DD8899DE83F7C3D00200000694015
:10B59000503E002078EB020040F7020028EB02004A
:10B5A00013B5334B3349044633481B1ADB081B04DD
:10B5B00043F003002246043C0190FBF705FA019892
:10B5C0000C2C22D8DFE804F0230E11332121141AA9
:10B5D00021072140400029490D2202B0BDE810405A
:10B5E000FBF7F2B926490522F7E726490622F4E7D8
:10B5F000254902B0BDE81040FBF7E2B90B22234910
:10B60000FBF7E2F9224B00221A7002B010BD21496B
:10B61000FBF7D6F9204B13211888FFF795FC30F083
:10B620000803F2D002B0BDE81040FBF7B9BC1B49DB
:10B63000FBF7C6F9184B1A884FF6FF739A42E4D10C
:10B64000174801F036FEEAE7FFF742FF15480022EF
:10B650004FF4CD71FBF79FFD08B1FBF7A1FC124839
:10B6600000221021FBF797FD0028CED0DAE700BFBB
:10B6700078EB020051F7020028EB020069F70200A4
:10B6800083F70200ABF70200D2F7020002F80200D3
:10B69000743500201FF802000E2B00204CF8020029
:10B6A00048390020A03D0020C83D0020013810B5D9
:10B6B000042843D8DFE800F0031C27303900204B72
:10B6C0001A7C002A3AD101221A749B7C172B1D4B3D
:10B6D0000BD9C8221C489A61FCF7DAFEBDE810407D
:10B6E000194832220021FCF77DBD4FF41672F1E7B4
:10B6F000134B1A7C12BB02221A749B7C172B114B22
:10B70000F3D96422E6E70E4B1C7CBCB903221A7401
:10B710000C4B4FF4FA72DDE7094B1C7C74B9042220
:10B720001A74084B4FF47A72D4E7054B1C7C2CB981
:10B7300005221A74034B4FF49672CBE710BD00BF7D
:10B74000503E0020B03E00202CFA02002DE9FF41BF
:10B750002B482C4D2C4F2D49BA7C2D4C2D1AED0821
:10B760002D0445F00300FBF72FF92A4A74231179C1
:10B77000237001236371A371E371237261722373D8
:10B780005179A3739279E37397F85D30E2720026E2
:10B79000BA7C2374601C1123A1726273ADF80E3061
:10B7A0006670A670E670267100F0BCFC1A4B1B4850
:10B7B0001B880DF10E02214602F052FB804645F037
:10B7C0000500174D14F8012B019029460136FBF7AF
:10B7D000FBF8112E0198F5D11249FBF7F1F8B8F1F9
:10B7E000130F87F8148004D80F4B23FA08F3DB07F4
:10B7F00002D44046FBF7D4FB04B0BDE8F08100BFA3
:10B8000028EB020078EB0200503E00207CF802009A
:10B8100051380020183E00200E2B0020102B002055
:10B820008CF802004CF9020021010A0037B5204BC8
:10B8300020482149214C224DC01AC008000440F084
:10B840000300FBF7BDF81F4A74231179237000230E
:10B850006370A370E370237161720123517992794F
:10B860006371A371E3712372E272A3730222E37323
:10B8700095F85D3022732374AA7CA1721123601C99
:10B880006273ADF8063000F04DFC0F4B0F481B887B
:10B890000DF10602214602F0E3FA1328287503D8B9
:10B8A0000B4BC340DB0701D4FBF77AFB03B030BD81
:10B8B00028EB020078EB020092F802005D370020CE
:10B8C000503E0020183E00200E2B0020102B0020A0
:10B8D00021010A0037B5204B20482149214C224D37
:10B8E000C01AC008000440F00300FBF769F81F4AC3
:10B8F00074231179237000236370A370E3702371A4
:10B9000061720123517992796371A371E37123729A
:10B91000E272A3730422E37395F85D3022732374FB
:10B92000AA7CA1721123601C6273ADF8063000F08E
:10B93000F9FB0F4B0F481B880DF10602214602F060
:10B940008FFA1328287503D80B4BC340DB0701D4AB
:10B95000FBF726FB03B030BD28EB020078EB0200BA
:10B96000A1F8020069360020503E0020183E002059
:10B970000E2B0020102B002021010A0037B5204B90
:10B9800020482149214C224DC01AC008000440F033
:10B990000300FBF715F81F4A742311792370002365
:10B9A0006370A370E37023716172012351799279FE
:10B9B0006371A371E3712372E272A3730322E373D1
:10B9C00095F85D3022732374AA7CA1721123601C48
:10B9D0006273ADF8063000F0A5FB0F4B0F481B88D3
:10B9E0000DF10602214602F03BFA1328287503D810
:10B9F0000B4BC340DB0701D4FBF7D2FA03B030BDD9
:10BA000028EB020078EB0200B1F802007535002047
:10BA1000503E0020183E00200E2B0020102B00204E
:10BA200021010A0030B50A4D0FCD87B001AC0FC41B
:10BA30002B682360074A0848012301A98DF80C30C0
:10BA4000FCF7DAFB08B1FBF7ABFA07B030BD00BF7B
:10BA50000CFA020069AF02002CFA0200084B0948F8
:10BA60000949C01A10B5C008084C0004224640F02D
:10BA70000300FAF7A9FF064BC3F8044510BD00BF49
:10BA800028EB020078EB0200BFF8020000005046ED
:10BA90000000014008B5FFF7E1FF054B1878FFF7FC
:10BAA00037F84FF08043B122C3F81C25FFF736FA70
:10BAB000863D002070B56D4C6D4D23686A7D013365
:10BAC0002360636801336360636901336361A36961
:10BAD000013BA361AB680133AB60236A013323628E
:10BAE000636A01336362CAB12B7DBBB166694FF4EF
:10BAF000FA7396FBF3F103FB11667EB95D4B5E486A
:10BB00005E49C01AC008000440F00300FAF75CFF69
:10BB10002B78012B09D1FFF719FE2677626940F6D1
:10BB2000B8339A4210DDFFF7F9F9022B02D1FFF783
:10BB30007DFEF2E7052B02D1FFF7CCFEEDE7032BEC
:10BB4000ECD1FFF71BFFE8E72B7C013B042B00F255
:10BB50008B80DFE803F0031533486D00AB7C172BB7
:10BB6000A36913D9962B06D10022BDE87040444842
:10BB70000021FCF737BBA369642B25D13222F4E7FF
:10BB8000AB7C172BA36901D9092B1FE0B3F5FA7F12
:10BB9000EAD0A369B3F5E17FF0D0A369B3F5AF7F35
:10BBA000E2D0A369B3F5967FE8D0A369C82BDBD0B8
:10BBB000A369962BE2D0A369632B07E0A369632BEB
:10BBC000D2DDA369642B4FD0A369312B4CDC00225A
:10BBD0002B481146FCF706FB00232B742848BDE8D0
:10BBE0007040FCF78FBCA369B3F5487FBCD0A36954
:10BBF000B3F52F7FC2D0A369B3F5FA7FB4D0A369A0
:10BC0000B3F5C87FBAD0A369C82BADD0A369642BA4
:10BC1000B4D0A369632B27DC002211461848FCF737
:10BC2000E1FA002316482B74FCF76CFCFFF732FF97
:10BC3000A369FA2B98D0A369C82B9FD0A369962B30
:10BC400092D0A369642B99D0A369312B0CDC00221C
:10BC500011460B48FCF7C6FA002309482B74FCF781
:10BC600051FC012385F8453070BD00BFB03E002077
:10BC7000503E002028EB020078EB0200D3F80200CF
:10BC80002CFA02001FB50B4A07CA01AB83E8070074
:10BC900009491846FEF7DCFE08B1FBF781F90748B1
:10BCA000FEF710FF08B1FBF77BF9FEF7FDFE05B0CC
:10BCB0005DF804FB20FA0200B9AF0200863D0020C7
:10BCC0001FB51B4C002320468DF80830FFF73AF9CA
:10BCD00044238DF8093033238DF80A30C0238DF8C2
:10BCE0000B3023798DF80C3063798DF80D3002A874
:10BCF000A3798DF80E30FFF723F90E48FFF722F9EC
:10BD00000D499DF80E409DF80C209DF80D304A72AB
:10BD10008B72CC7209480A490094401AC00800048A
:10BD2000084940F00300FAF762FE04B010BD00BFFE
:10BD30001F3E0020183E0020002B002078EB020060
:10BD400028EB0200F2F8020070B5B64BB64DB749C9
:10BD5000ED1AED08B4B02D0445F005000190FAF796
:10BD60002FFEB3490198FAF72BFEB0490198FAF774
:10BD700027FEFFF76DFB4FF480410020FAF786FCA9
:10BD800008B1FBF70DF9FAF7BFFBAA48FDF74AF82F
:10BD9000FFF748FEFDF75CF808B1FBF701F9FBF788
:10BDA000BDF908B1FBF7FCF8A34AA448A44C012153
:10BDB000FBF7E6F90121A34AA348FBF7E1F900F0FC
:10BDC000F9F94FF08043A149D3F81C3584F8443089
:10BDD0000320FFF735F808B1FBF7E2F809A90020C6
:10BDE000FFF78AF808B1FBF7DBF8FCF729F808B190
:10BDF000FBF7D6F802F0C8F808B1FBF7D1F800233A
:10BE000009A90120099302F091F908B1FBF7C8F8DC
:10BE100009A802F04BFA08B1FBF7C2F80120FFF7BE
:10BE20009FF808B1FBF7BCF8FFF74AFF4FF08043DB
:10BE30008748D3F80034A364FF23237511238DF8BA
:10BE4000183002F0FAFD06AE82B281493046FFF7A3
:10BE50007FF808B1FBF7A4F80023ADF828301023D1
:10BE6000ADF824303C23ADF8263009A84FF4C87350
:10BE7000ADF82A30FFF76AF808B1FBF791F8FFF741
:10BE800001FB744B7448099309A901F05FFE08B1E6
:10BE9000FBF786F8714B72480693314601F066FF56
:10BEA00008B1FBF77DF8FE238DF80F302023ADF8A5
:10BEB0001430AC222823002109A8ADF8163002F076
:10BEC00067FD05228DF827200DF10F0202230A924B
:10BED00005AA8DF824301192ADF81C304D228DF852
:10BEE000603001234021ADF810208DF8A030592298
:10BEF0004FF49673CDE92B13ADF81820594B5A48DF
:10BF0000219604AA09A90892329301F010F808B109
:10BF1000FBF746F8544E0121304601F005F8534B2B
:10BF20001422002109A81E6002F032FD4FF4F02314
:10BF30004FF4A032CDE90A2303238DF830304C4B67
:10BF40000E9309A84B4B0F9301F0D2FA08B1FBF7FF
:10BF500027F8494A49480021FBF712F908B1FBF7D5
:10BF60001FF8384A38480121FBF70AF908B1FBF7F6
:10BF700017F845F003004249FAF722FD00F0A0F857
:10BF8000FDF7C0FC002047F23053E070E360FEF79D
:10BF90004BFF08B1FBF704F894F8442062BB394822
:10BFA0004FF4CD71FBF7F7F808B1FAF7F9FF36480F
:10BFB00000221021FBF7EFF808B1FAF7F1FF334B3D
:10BFC000012222701A77052000225A61FFF76EFBCA
:10BFD000FAF7ACFB08B9FBF749FF94F84530012BA1
:10BFE000F6D12848FBF7EFF82748FBF7ECF84FF0BD
:10BFF00080430222C3F81C25FFF744FE244B187827
:10C00000FEF786FD00224FF061712248FBF7C3F86E
:10C01000FEF7A8FF08B1FAF7C3FFFFF759FA1E4C65
:10C020003CE000BF28EB020078EB02000FF90200B1
:10C030004EF9020065B00200B5BA020064FA0200CF
:10C04000503E002061B0020060FA0200A1B502007B
:10C05000002B0020D9AF02000C3E0020C1B202002C
:10C06000102B002009B1020048390020283E002092
:10C07000C5B302004DB40200DDAF020070FA020049
:10C080007DF90200A03D0020C83D0020B03E002008
:10C09000863D0020303E00206C35002023680133AF
:10C0A0002360FAF743FB0028F8D1FBF7DFFEF5E742
:10C0B000024BA0F5064053F820007047E4FB020055
:10C0C000014B03221A617047B03E0020F0B5114BBE
:10C0D00087B002AC06460A4603F1100C27461868E2
:10C0E0005968254603C5083363452C46F7D10A48ED
:10C0F0000A4B0B4901921B1ADB081B0443F0030097
:10C10000FAF75EFC019A3946304600F0B3FB07B0FF
:10C11000F0BD00BF89FA020028EB020078EB0200B4
:10C1200074FA0200F0B5114B85B06A46044603F17B
:10C130001007164618685968154603C50833BB42F0
:10C140002A46F7D10A4D0A4A2046314600F07CFBC8
:10C15000234605F110042A4603CAA242186059601A
:10C16000154603F10803F6D105B0F0BD89FA0200C7
:10C170009C3E0020014B00221A7070473C3F00207B
:10C1800070470000014B01221A7070473C3F0020AD
:10C19000054B5B78012B05D1044A042082F843301B
:10C1A000FFF784BA704700BFD83E0020503E002001
:10C1B00070470000104803784FF0A04203F5E07389
:10C1C0000C2142F82310437803F5E07342F8231062
:10C1D0000A4B19229A6028229A70094B094ADA619F
:10C1E000094A1A62094A9A64094ADA6405229A607D
:10C1F000084A5A62704700BF342B0020303F0020AD
:10C20000D83E002075C1020081C1020091C1020028
:10C21000B1C1020085C1020008B50D480D4B0E49A1
:10C22000C01AC008000440F00300FAF7C9FB0B4B2A
:10C2300001221A700A4B1A7700225A61094B1B78A7
:10C240000BB9FFF735F9BDE808400120FFF72EBA1A
:10C2500078EB020028EB020020FC0200503E002098
:10C26000B03E00207435002008B50E480E4B0F4933
:10C27000C01AC008000440F00300FAF7A1FB0C4B01
:10C2800002221A700B4B01221A7700225A610A4BC4
:10C290001B780BB9FFF70CF9BDE808400220FFF747
:10C2A00005BA00BF78EB020028EB02002EFC02006A
:10C2B000503E0020B03E00207435002008B50E48E6
:10C2C0000E4B0F49C01AC008000440F00300FAF7F3
:10C2D00077FB0C4B03221A700B4B01221A770022BA
:10C2E0005A610A4B1B780BB9FFF7E2F8BDE808402A
:10C2F0000320FFF7DBB900BF78EB020028EB020058
:10C300003DFC0200503E0020B03E0020743500206D
:10C3100008B50B480B4B0C49C01AC008000440F08C
:10C320000300FAF74DFB094B00225A61084B01222A
:10C3300083F84320BDE808400420FFF7B7B900BFE9
:10C3400078EB020028EB02003DFC0200B03E00202A
:10C35000503E00202DE9F047414C424FDFF8088164
:10C36000DFF80891DFF808A1002625464FF0A0432A
:10C3700017F8012BD3F81035D340DB074CD4012339
:10C380002370A378012B0ED0637883B963690133DE
:10C390006361E36920469847012363706368013352
:10C3A00063602C340EB1BDE8F0870126DEE7E36858
:10C3B0002BB1E278934202D8A36A204698472B6BB0
:10C3C000142B03D16B7823BBFFF726FF99F80220CB
:10C3D0006368B3FBF2F102FB1133002BDCD1E2788E
:10C3E0000132E270EA78511E042905D8052ACAF8FC
:10C3F000143001D1FFF762FFA368002BCCD0E278A4
:10C400009342C9D8A3690133A3610123A370636A6E
:10C41000C0E7FFF77DFFD9E76378012B0CD1BEB9E8
:10C420006B68023B612B0FD898F843300BB9FFF7CC
:10C430001BFF236A204698470023237063606370C4
:10C44000E370A3702361ACE7C5E900662E61F0E7F5
:10C450002B6B182B9EBF0023C5E90B33EB63E8E77A
:10C46000D83E0020342B0020503E0020303F0020DA
:10C47000B03E0020274B284A1B6873B503F110011A
:10C48000187810705878507098789070D878D0706C
:10C4900004338B4202F10402F2D1204B2048214C9C
:10C4A00004211A6801928D0714D1C2F30746C2F322
:10C4B0000725865D8DF80560160ED2B2455D825C5B
:10C4C0008DF807208A08865DA25C8DF806606A40B8
:10C4D0008DF8042013F80C2C9DF804506A401A7152
:10C4E0009DF8055013F80B2C6A405A719DF80650C0
:10C4F00013F80A2C6A409A719DF8075013F8092C1A
:10C5000001316A402C29DA7103F10403C9D102B068
:10C5100070BD00BF403F0020443F0020503F00203E
:10C520004DFE02004EFC02000B4B1968F0B50B4E9D
:10C530000A1D00011431131F35181C7815F8017BF2
:10C540007C4003F8014B9342F7D11A1D8A4200F157
:10C550000400F0D1F0BD00BFF43F0020443F0020B4
:10C56000084B09481B6810B5191D002213F822401A
:10C57000045D03F822400132042AF7D101338B42D3
:10C58000F3D110BDF43F00204DFE02000D4B1B689F
:10C5900059795A785970597A5971597B5972997ADF
:10C5A0005A739A789970997B9A729A799971D97B12
:10C5B0009A73DA78D970D97AD973D979D972DA714C
:10C5C000704700BFF43F0020C30903EB430303EBB4
:10C5D000C30383EA4000C0B270470000084B09481B
:10C5E0001B6810B5191D002213F82240045D03F8E2
:10C5F00022400132042AF7D101338B42F3D110BD1E
:10C60000F43F00204DFD02000D4B1B68597A5A7B08
:10C6100059735979597259785971997A5A709A7827
:10C620009970997B9A729A799971D9799A73DA7813
:10C63000D970D97AD971D97BD972DA73704700BFB2
:10C64000F43F00202DE9F84F0020FFF76DFF214F48
:10C650000124FFF785FFFFF799FF3A6802F1100AFE
:10C6600092F800905578917892F8038089EA050055
:10C6700081EA080B8BEA0006FFF7A6FF89EA0000B3
:10C680007040107085EA0100FFF79EFF684070401F
:10C6900050705846FFF798FF48407040907089EA04
:10C6A0000800FFF791FF88EA00004640D670043288
:10C6B0009245D5D120460134E4B2FFF735FF0A2C6C
:10C6C000C7D1FFF74DFFFFF761FF2046BDE8F84FE8
:10C6D000FFF72ABFF43F00202DE9F04F0A2089B070
:10C6E000FFF722FF0926FFF78FFFFFF777FF30469E
:10C6F000FFF71AFF4E4B196801F11003069391F8EA
:10C70000009091F801808F7891F803A04846FFF7D8
:10C710005BFF0090FFF758FF0190FFF755FF83463E
:10C720004046FFF751FF0246FFF74EFF0290FFF72A
:10C730004BFF05463846FFF747FF0390FFF744FFDE
:10C740000790FFF741FF04465046FFF73DFF049076
:10C75000FFF73AFF0590FFF737FF009BDDF81CE07D
:10C760009C46019B8CEA030C8BEA0C0C029B82EA30
:10C770000C0C8BEA02025A40039B6A405A40059B0C
:10C7800062405A40424089EA0202019B7A408AEAAA
:10C7900002024A7083EA0B02039B6A405A4082EA13
:10C7A0000E02049B62405A40424089EA020288EA33
:10C7B00002028AEA02038B70009B83EA0B0B029B46
:10C7C00085EA0C0C83EA0B0B8EEA0C0C049B84EAC2
:10C7D0000C0C85EA0B0580EA0C0C6C4088EA0C0C0A
:10C7E0005C40059B87EA0C0C8AEA0C0C83EA040A7D
:10C7F00080EA0A0089EA000988EA090887EA080746
:10C8000081F800C0CF70069B04318B427FF477AF74
:10C81000013E16F0FF067FF466AFFFF7F5FEFFF767
:10C82000DDFE304609B0BDE8F04FFFF77DBE00BF2A
:10C83000F43F00204B1E01380F3113F8012F00F890
:10C84000012F8B42F9D1704738B50D46014610468D
:10C850001446FFF7EFFF054B1C60054B1D60FFF70B
:10C8600009FEBDE83840FFF7EDBE00BFF43F0020F1
:10C87000403F002038B50D46014610461446FFF7EC
:10C88000D9FF054B1C60054B1D60FFF7F3FDBDE8AC
:10C890003840FFF721BF00BFF43F0020403F002099
:10C8A0000369C26893429CBF80681B18013B981AB9
:10C8B00070472DE9F843D0E902940546A9EB040836
:10C8C0004068904520440F46144404D902F037F8DC
:10C8D000EC60BDE8F8834246A4EB090402F02FF8AF
:10C8E0006868224607EB0801F0E72DE9F843C568C0
:10C8F0000646894617464FF000083469B3687068E9
:10C90000A54228BFE418013C621B5C1BBC4228BF47
:10C910003C46944228BF144649462844224602F029
:10C920000EF8B3682544AB4208BF00253F1BA04466
:10C93000A144F560E1D14046BDE8F88310B5114C43
:10C94000114AA2610223C4E90433104BE361A264DB
:10C950004FF400730E4A0F492362E2640023102251
:10C96000E01DA3626362E362A3656365E36522651C
:10C9700002F041F80849204602F03DF82023A37157
:10C9800010BD00BFF83F00204DFF02008040002096
:10C990007040002056FF02005AFF020070B5164B8F
:10C9A000182400FB04451D4404FB00331646DC6AD2
:10C9B000012C0ED0022C18D0E4B92846FFF770FFE6
:10C9C000864204D832462846FFF773FF3446204695
:10C9D00070BD2846FFF764FF8642344628BF0446F0
:10C9E00022462846FFF765FFF1E72846BDE870407C
:10C9F000FFF77BBF0024EAE7F83F0020FFF79EBF68
:10CA00006DDF704779DF70477DDF704764DF704707
:10CA10002DE9F04F85B000250E9CBDF83CB0B4F870
:10CA200000A00191074690461E46A9463A884A450D
:10CA30000DDC45B12388013BA3EB0A039BB2FF2B1E
:10CA40003AD806F80A30002005B0BDE8F08F7A68C1
:10CA500052F82900039000220DF10B0103A8FFF703
:10CA6000D5FF0028F0D19DF80B20424521D1228826
:10CA7000002D14BF0020022002EB0801014459459B
:10CA80001ADC3DB9013292B2019B2280B354228854
:10CA90000132228022880DF10B01324403A8FFF7F6
:10CAA000B5FF0028D0D121889DF80B200A442280B0
:10CAB000012509F10109B9E70C20C5E72DE9F3418A
:10CAC000089FBDF824801546CDE90078022204466F
:10CAD0001E46FFF79DFF50B93346102229462046D7
:10CAE000CDE9087802B0BDE8F041FFF791BF02B090
:10CAF000BDE8F0812DE9F04F00231788138090F8EE
:10CB00002D3085B006460D4614465BB3082F01D87C
:10CB10000C2028E102A8FFF773FF002840F02381D2
:10CB20002388DDF809100822EA54238801339BB2D8
:10CB30001B222380EA54238801339BB2EA18238006
:10CB4000E950BDF80D30938023889DF80820063306
:10CB50009BB212F0FE0218BF01222380EA54238800
:10CB600001332380B378FBB123880433BB42CFD891
:10CB700002A8FFF747FF002840F0F5802388032232
:10CB8000EA54238801339BB219222380EA54238874
:10CB9000BDF8082001339BB2E9182380EA54120A39
:10CBA0004A70238802332380F2789AB12388D91CF3
:10CBB000B942ADD80221E954238801339BB2012147
:10CBC0002380E95423880B449BB22380EA542388B2
:10CBD0000B4423807268AAB12388D91CB94297D824
:10CBE000022192F90020E954238801339BB20A21E3
:10CBF0002380E954238801339BB22380EA5423889D
:10CC0000013323803389002B40F0A180338A5BB14C
:10CC1000CDE900472B460722032106F11000FFF75C
:10CC20004DFF002840F09F80338B5BB1CDE900477A
:10CC30002B461522142106F11800FFF73FFF0028AC
:10CC400040F09180326A002A40F09080D6F824802B
:10CC5000B8F1000F30D0B8F804302188981C8A1C35
:10CC60000244BA423FF654AFFE283FF651AF0333B9
:10CC70006B54238801339BB2FF222380EA5423881C
:10CC800001339BB22380B8F80020EA54E918120A55
:10CC90004A702088023080B22080B8F804205AB14F
:10CCA000D8F8081000296BD0284401F048FE2388EA
:10CCB000B8F804201344238096F82C30002B40F061
:10CCC0009880307800284ED03388012B58D02288A5
:10CCD00002F1020CBC453FF61BAF012805D1737869
:10CCE000023313449F42FFF413AF023FBF1ABFB297
:10CCF00002A905EB0C00ADF80870FFF785FE90BBAC
:10CD00003178BDF80830022900F0B98072789A4273
:10CD100002D39F4280F0B180012940F0B280974257
:10CD200093B2C0F0AE80ADF808300821BDF80830ED
:10CD3000FE2B3FF6EDAE22880133AB542288013240
:10CD400092B22280A9542288134423800BE0CDE9BB
:10CD500000472B460622022106F10800FFF7AEFE2F
:10CD600000283FF453AF05B0BDE8F08FB4F800C021
:10CD70000CF10603BB423FF6CBAE1188052901D862
:10CD80000720F0E76FF4486E01EB0E039BB24FF201
:10CD90007D3E7345F4D95388052BF1D96FF4486073
:10CDA000181880B27045EBD94FF6FF70814201D060
:10CDB0009942E5D8052305F80C30238801339BB24E
:10CDC00012212380E954238801339BB223801188E8
:10CDD000E954E818090A4170238802339BB2238082
:10CDE0005288EA54E918120A4A70238802332380D1
:10CDF0002CE7B36A002BC3D04FF000084FF00C0AA9
:10CE00004FF0160BB16A5FFA88F20AFB02F201EBEF
:10CE10000209B9F80430981CFE283FF679AE208844
:10CE200003332B54238801339BB2238005F803B0CE
:10CE3000238801339BB223808A5AEA54E918120AE4
:10CE40004A702088023080B22080B9F804205AB19C
:10CE5000D9F80810002993D0284401F070FD2388E8
:10CE6000B9F804201344238096F82C2008F1010817
:10CE70005FFA88F39A42C5D823E7092156E79F4213
:10CE8000FBD2ADF8087050E730B5C8B1F2B100245C
:10CE9000651C8D4206DA1588A54212D805196D78F1
:10CEA0009D420ED1A14211D9005D48B1013880B236
:10CEB00030B10234A3B210FA84F4A14206DB13802D
:10CEC00030BD055D01352C44A4B2E1E70020F7E751
:10CED00013B513460022ADF806200DF106020446F4
:10CEE000FFF7D2FF10B1BDF80630E01802B010BD58
:10CEF00072DF704773DF704774DF704738B5012207
:10CF000004460D46B0F81414D0F81004FFF7E0FF03
:10CF100000B1057004F13C0204F5826104F1540093
:10CF2000BDE83840FFF7E4BF80F830107047F8B52F
:10CF300004460F46002973D0002871D091F87A304A
:10CF40001BB191F89830002B6CD1D7F8A030042B8E
:10CF500068D0D7F89C30042B64D04FF0000C84F8D4
:10CF600002C007F178060FCE251D0FC50FCE0FC5E5
:10CF700096E8070085E8070084F830C0D7F8A430A9
:10CF80006363D7F8A830A36304F582624FF6FF739A
:10CF9000C4F826C4A4F82434C4F82024C4F829C44E
:10CFA00022780AB984F8543094F82430002B14BF46
:10CFB000EE231F2304F15501C4F81014A4F814340F
:10CFC00004F214423846FFF795FD40BB94F8243034
:10CFD000002B14BFEE231F2304F23121C4F81814D0
:10CFE000A4F81C3404F21C4207F13C00FFF782FD58
:10CFF000A8B9A369A4F848304FF480730125A4F8B8
:10D00000503063692064014684F83C50636404F145
:10D010003C0204F15400FFF76BFF00B92570F8BD26
:10D020000E20FCE70720FAE7F8B5077804460D461E
:10D03000002F00F007810023C0F82634C0F82934FF
:10D04000C388817000F226460BB1012903D0E37931
:10D0500043B1022D06D1636BABB1012284F82D24BC
:10D060000820984704F2274304F22D4113F8012BBE
:10D0700012B99942FAD117466B1E032B4ED8DFE83E
:10D0800003F0050B0F1284F82D34EBE7A3791BB1E5
:10D0900094F8243003B95FB9E3790BB1002F3FD185
:10D0A000237A002B3ED1637A002B0CBF0025042588
:10D0B000636BA570002B37D0033D012D34D8627906
:10D0C00092B394F82E247ABB84F83024012284F899
:10D0D0002F240720984704F13C05182200212846F8
:10D0E00001F056FCE26A531E0121022B28BF0A46BA
:10D0F00084F8512094F8242084F83C1032B1A36ABB
:10D10000581E022828BF0B4684F85230A378042BFF
:10D110001CD8DFE803F0780D23365A000025C7E756
:10D120000225C5E70325C3E7002384F82F34D2E79F
:10D13000012384F831300023C4E91063C4F820349B
:10D14000022384F83C308023A4F84830A378002BD5
:10D150005DD1636B002B71D100206EE00223002AA9
:10D1600084F8313014BF0723032384F83C3023694B
:10D17000A4F848300023C4F82034E36826646364CC
:10D18000E4E763696364A369A4F8483012B1062335
:10D1900084F83C306379B3B194F82E349BB994F899
:10D1A000303483B1022384F8503004212046FFF745
:10D1B000A5FE0028CAD1052384F8313004F5826326
:10D1C000C4F82034C2E70323F6E7E3696364236A03
:10D1D000A4F8483012B1062384F83C30637983B157
:10D1E00094F82E346BB994F8303453B1022384F898
:10D1F000503004212046FFF781FE0028A6D10623E7
:10D20000DAE70423D8E7002384F831309EE794F866
:10D210005330D4F8201443F0100384F853302A46D6
:10D2200004F15400FFF764FE38B994F8301094F814
:10D230005400FFF75FFE00288BD0F8BD94F8310052
:10D24000984789E70820F8E70388112B10B50C46AA
:10D250000AD0262B1FD0102B05D1C37B012B02D166
:10D260008388A1F8243410BD0022838881F82E24FD
:10D27000B1F824249A42F6D10B79002BF3D1012185
:10D280002046FFF7D1FE0028EDD0A36B002BEAD09B
:10D29000BDE810401847037A013B012BE3D8897899
:10D2A00005230131B1FBF3F303EB8303C91AC9B2C0
:10D2B000E6E738B5044690F85400FFF71DFE012359
:10D2C00084F82E34002384F8303484F8503006215A
:10D2D0002046FFF713FE054638B9A1782046FFF730
:10D2E000A3FE10B1A36B03B19847284638BD75DF84
:10D2F000704776DF70477ADF70477BDF704700004A
:10D30000034B1A8882420CBF18460020704700BFAA
:10D310009C420020024B9B6903B11847704700BF35
:10D320008042002073B585B22846FFF7E9FF044626
:10D3300038B3174E027A337B9A420CD200F10A01BD
:10D340002846FFF7D4FFF0B111281AD002B0BDE88B
:10D350007040FFF7DFBF00230372337C43B13B21F2
:10D360002846FFF7C6FF30F0080301D0FFF7D2FFD1
:10D37000736933B100228DF80420ADF8065001A87E
:10D38000984702B070BD237A01332372F9E700BFDA
:10D390008042002037B50B46497A0F4A79B9D2E965
:10D3A00001141D7A0246002D18BF21465868F9F76E
:10D3B000F2FE78B103B0BDE83040FFF7ABBF00210B
:10D3C0001972536933B10122ADF806008DF80420BB
:10D3D00001A8984703B030BD804200204B880288E6
:10D3E0009A4212D842889A420FD380888B8840F2A2
:10D3F000F311884294BF021A421A9A4205D808448F
:10D40000984234BF00200120704700207047000080
:10D410000388122B70B5014659D004D8102B1ED0AA
:10D42000112B44D070BD502BFCD12F4BC288DB890F
:10D430009A42F7D1038A022BF4D186883046FFF74F
:10D440005FFF05460028EDD001F1120000F07FF9E2
:10D4500038BB6868F9F7B7FE0028E3D009E0C37B62
:10D46000012BDFD14FF6FF70FFF74AFF054620B9C9
:10D470000420BDE87040FFF74DBF1C4A8E8806802F
:10D48000002303721368C0F80A305368C0F80E30E6
:10D4900010310A30FFF7A2FF134B6872DB89002BB3
:10D4A000C0D129463046BDE87040FFF773BF808881
:10D4B000FFF726FF04460028B4D04068F9F783FE42
:10D4C00008B1FFF727FF4FF6FF732380AAE786888E
:10D4D0003046FFF715FF05460028A3D008310A3073
:10D4E000FFF77CFF6872DCE780420020B04200203A
:10D4F000F8B5064648B305460FCD154F3C460FC458
:10D5000095E8070084E807003068124C3C60B0B131
:10D51000FFF7F1FEC0B93268136823605368636097
:10D520000D480E4A4FF6FF7303800D4B40F8043F41
:10D530000021F9F725FE002818BF032004E020464B
:10D54000FFF7DBFE0028EBD0F8BD0E20FCE700BFA4
:10D5500080420020B04200209C42002025D30200DF
:10D56000B84200200AB1FAF725B9FAF72CB973B519
:10D570000191019C06466CB100252C46294601A864
:10D58000FAF72BF918B106EB440301349D800135FD
:10D59000142DF3D13046346002B070BD2DE9F04750
:10D5A00003888488103B8CB005460A2B21D8DFE81D
:10D5B00003F0064020202020202020654700DFF8CF
:10D5C000E880D8F80830DB430093D8F804106846A8
:10D5D000FAF73BF9009901A8FFF7C9FF0DF1080917
:10D5E0000027019B9F4207D3132C12D90420F9F77F
:10D5F000D7FC0CB0BDE8F08739F802AB0026013645
:10D60000514608EB8600FAF7DEF81E2EF7D10137F7
:10D61000E7E71F482146FAF7CDF81E482146FAF7FA
:10D62000C9F8EB7B022BE4D11B482146FAF7C2F87C
:10D63000DFE7174821460CB0BDE8F047FAF7C3B85A
:10D64000027A16483F2A4FEA1215214694BF00225B
:10D650000122FFF787FF022D94BF0022012210480C
:10D660002146FFF77FFF012D0E4894BF00220122C3
:10D6700021460CB0BDE8F047FFF774BF037A002BDA
:10D68000B7D1427A0548C2F3C0022146F1E700BF94
:10D69000E0420020DC420020E4420020F042002072
:10D6A000EC420020E8420020D84200201328014626
:10D6B00002D80248FAF791B800207047DC420020F7
:10D6C00010B50446FFF7F2FF002814BF20461420CF
:10D6D00010BD70B50546164608460AB90E2070BD45
:10D6E00000231360002DF9D02B68002BF6D0EB88B7
:10D6F00013F003040ED1FFF7E3FFC0B214280BD0E0
:10D700002B7983420AD9EA882B6800FB023030600B
:10D710002046E4E70720E2E70520E0E70420DEE713
:10D72000AADF7047002301380B70042806D8DFE811
:10D7300000F00306080A0C0011230B707047212328
:10D74000FBE73123F9E71223F7E72223F5E7008807
:10D7500000F001007047F0B58B7891B00C46012BBA
:10D7600038BF012300278DF80E3005460B88607CFA
:10D77000ADF80C306946ADF800708DF80270FFF717
:10D78000D1FFA07C0DF10101FFF7CCFF1646237BF2
:10D79000E27B217D43EAC203227C43EA02139DF827
:10D7A0000220B94222F0190203F0190314BF02212A
:10D7B0000121134361F342031C22394609A88DF865
:10D7C000023001F0E5F8637B13F0300F14D00DF157
:10D7D0000901E07CADF808708DF80A70FFF7A2FF30
:10D7E00011238DF808309DF80A30012102AA61F357
:10D7F00042038DF80A300E92637B8DF82430A37BB0
:10D800008DF825300023CDE90633089303AB04934C
:10D81000A388ADF81C30A368CDF814D01BB1E28802
:10D82000ADF818200893A36973B301A90022ADF8DD
:10D8300004208A701A88ADF82C205A88ADF82E2062
:10D840005A680D91187B0A92FFF76CFFA3690DF1DE
:10D850000501587BFFF766FFA3699A7A197A41EAB6
:10D86000C201DA7A9B7B41EA02119DF80620002B67
:10D8700001F0190122F0190214BF02230123114300
:10D8800063F342018DF80610E36903B10C9333464C
:10D8900004AA09A92846FFF743FF11B0F0BD90DFA5
:10D8A0007047A5DF7047B5DF704700007FB50023E4
:10D8B000ADF80810ADF80A106A4602A90646ADF8A0
:10D8C0000C30ADF80E300093ADF80430FFF7E7FFF1
:10D8D000054600B3114B124CE41AE408FAF752FB68
:10D8E000240444F0010403460E4932462046F9F769
:10D8F00074F8BDF80020BDF8023052EA030103D0ED
:10D9000009492046F9F769F8BDF804201AB107491A
:10D910002046F9F759F8284604B070BD28EB0200FC
:10D92000A0EB020061FF0200ABFF0200EAFF020071
:10D9300080B14FF0F7130360FB230371F723C3801B
:10D940001723038141F6FB32002301614381828169
:10D95000184670470E20704730B1A1F11703E02B35
:10D9600004D80180002070470E20704707207047C0
:10D9700013B5034680880C46B8B91A88242A00F0EB
:10D980009C8014D8112A74D0232A00F0A780102A72
:10D990003ED0A37A4BB1E1880020FFF782FF002838
:10D9A00040F0A2804FF48073638102B010BD3A2A28
:10D9B00068D0552AEDD1DB88C988A072172B38BFF3
:10D9C00017238B4228BF0B462381FFF76CFF60B102
:10D9D000FAF7D8FA4E4B4F4902464F481B1ADB085C
:10D9E0001B0443F00100F8F7EFFFE27A002AD0D1E0
:10D9F0002369002BCDD040F67721ADF80220228993
:10DA0000ADF80010ADF80420694620469847C0E7FD
:10DA1000DB7B0A790A73012B13D0022B14D0E18827
:10DA200023898B4205D20020FFF73BFF70B9012309
:10DA3000E372217B637B8B42ABD20020FFF736FF82
:10DA4000A7E70B88E380EAE74B88FBE7112802D1C0
:10DA50000123A372EDE7FAF795FA2D4B2F49024601
:10DA60002D481B1ADB081B0443F00100F8F7ACFF3C
:10DA7000DFE7F723CB8017230B8141F6FB33488187
:10DA80008B8186E75B89CA88934228BF1346172B90
:10DA90000A6938BF17230B8162B1C97A51B140F6C8
:10DAA0007721ADF80010ADF80200ADF804306946FA
:10DAB00020469047002363816BE71A7A0B694A730B
:10DAC000002B3FF466AF4DF67A218DF80500ADF8D6
:10DAD0000010ADF802008DF8042095E7197A237B39
:10DAE000994228BF1946A9E711283FF45EAFFAF71B
:10DAF00049FA074B0949024607481B1ADB081B0471
:10DB000043F0010002B0BDE81040F8F75DBF00BF70
:10DB1000A0EB02007100030028EB020040000300AC
:10DB2000B0DF704766DF704710B5002104464088BB
:10DB3000FFF7F8FF034608B9237210BD112801D181
:10DB40000123F9E76368BDE81040184760B159B197
:10DB50000378DE2B0AD00B684360DE2303704FF698
:10DB6000FF734380002070470E20704708207047E5
:10DB700028B10378DE2B04D14180002070470E20AD
:10DB8000704708207047F0B5054685B00C4600295F
:10DB900042D0002840D00B78DE2B3DD182884B88C4
:10DBA0009A4204D10B7A13B10846FFF7BDFF2B88C8
:10DBB000112B33D0512B0FD0012B2DD12B7A012BD0
:10DBC0002AD1A9886288914226D12046237205B0C5
:10DBD000BDE8F040FFF7A8BFAE886388B3421BD111
:10DBE000AF79022F18D1AD7B2B1F022B14D8002147
:10DBF0001022684600F0CCFE052D18BF4FF4C0730C
:10DC00006946304618BFADF804308DF80070FFF754
:10DC100087FF08B16368984705B0F0BD6388AA889C
:10DC20009A4204BF4FF6FF736380F5E7A8DF7047A1
:10DC3000ADDF7047AEDF704762DF7047F0B5054675
:10DC40008BB00C4600295FD000285DD00388502B94
:10DC500035D0572B6CD0102B56D1818860690026A7
:10DC600001AA0196FFF735FD02232189A888ADF8A6
:10DC70000A6002AACDF80CD0ADF80830FFF7D8FF43
:10DC8000002841D1A369002B3ED00398FFF75FFD28
:10DC9000002839D0019E0EB10123337018220021D3
:10DCA00004A800F075FE02238DF81030AB88ADF8A3
:10DCB0001830A3690594079604A8984724E0818842
:10DCC000606902AAFFF705FD1822002104A800F0F0
:10DCD0005FFEAB882189ADF81830EB88029A059475
:10DCE0009942079217D12E8A022E14D162B105F102
:10DCF0001200FFF72CFD029B40B101221A708DF833
:10DD00001060A369002BD7D10BB0F0BD18700323AE
:10DD10008DF81030F5E7A2899A42F5D1A369002B5E
:10DD2000F2D005F1120208922A8AADF82420C3E746
:10DD30008188606902AAFFF7CCFC01460028E3D184
:10DD4000029F3B78002BDFD0A669002EDCD0182282
:10DD500004A800F01DFE01238DF81030AB88059457
:10DD6000ADF81830079704A8B047CDE7F0B53A4BA7
:10DD70008FB002AD04460A4603F1100C2F46186816
:10DD800059682E4603C6083363453546F7D1002C43
:10DD90005FD0002A5DD01368A36121463846FFF7A3
:10DDA0004BFF002853D12246012512F8023B8DF883
:10DDB000063001A92846ADF80450FFF737FF0028C8
:10DDC00045D10146202206A800F0E2FD22460223AA
:10DDD000ADF8183012F80C3B8DF81A30BDF824302D
:10DDE0001E4E6088079623F44F6323F00F0343F41D
:10DDF00040632B4306A9ADF824308DF829508DF8E7
:10DE00002A50FFF7A8FC10BB0146202206A800F00C
:10DE1000BFFD22460323ADF8183012F8043B8DF8FD
:10DE20001A30BDF824306088079623F4875323F016
:10DE30001F0343F480532B43ADF8243006A940F26E
:10DE400001138DF82950ADF82A30FFF784FC0FB08C
:10DE5000F0BD0E20FBE700BFB5000300F400010099
:10DE6000F0B50F4687B016461C46054610B340690C
:10DE700001AA1946FFF72DFCD0B94FF6FF739C425B
:10DE80001AD0019BC3B11B78C3B13388F42B17D8C8
:10DE9000AB88CDF80B008DF80F00ADF8083002A963
:10DEA00001232046CDE904678DF80A30FFF7C2FE52
:10DEB00007B0F0BD0E20FBE70520F9E70820F7E7E3
:10DEC0000720F5E710DF704711DF704713B50446F0
:10DED00009496846F9F7FBFF019808B902B010BD7F
:10DEE000D0E900212046904718B16846F9F7F9FFBC
:10DEF000F2E71120F2E700BFD400030013B5044697
:10DF000007496846F9F7E3FF019B0BB902B010BD62
:10DF10002046D3E9002190476846F9F7E2FFF3E78E
:10DF2000EC000300084B9A6822B11A6822F48002C0
:10DF30001A607047054B4FF48002C3F88020BFF38E
:10DF40004F8FBFF36F8F7047E431002000E100E096
:10DF50000B4991F816335A09EC231341DB0706D518
:10DF6000084B9A683AB94FF480030B60704742F24D
:10DF70000200F9F715B81A6842F480021A60704777
:10DF800000E100E0E4310020F7B5194F3C7864BBB4
:10DF9000184E012520463570FFF798FF112821D033
:10DFA0002046FFF7ABFF144B8DF803401868019033
:10DFB0000DF10300F9F7DCF9104901A8FFF782FF22
:10DFC0000446B0FA80F0400938709DF80300F9F774
:10DFD000F3F93CB90A4B34701C70FFF7B9FF2846BF
:10DFE000FFF78CFF204603B0F0BD0824FAE700BF1E
:10DFF0005543002054430020CD000300BD6F0200B4
:10E0000056430020F7B5154F3B781BB3144E012043
:10E010003070FFF75BFF11284FF000051CD0022085
:10E02000FFF76CFF0DF107008DF80750F9F7A0F925
:10E03000FFF74AFF04469DF807003D70F9F7BCF969
:10E040002CB903203470FFF76DFFFFF757FF204610
:10E0500003B0F0BD0824FAE72C46F8E7554300204A
:10E0600054430020054B1B7833B1054B1B780BB193
:10E07000FFF7C8BFFFF788BF082070475443002050
:10E0800055430020014B1878704700BF55430020CE
:10E0900007B508496846F9F71AFF019B13B903B0A1
:10E0A0005DF804FBD3E9002090476846F9F719FFB3
:10E0B000F3E700BFE0000300FFF7EABF60DF70474F
:10E0C00069DF704761DF704730B5134DADF5017DF5
:10E0D0004FF4FA740DF1020103A8ADF80240FFF706
:10E0E000F1FF70B9294601A8F9F7F1FE029B002B58
:10E0F000F0D003A8D3E90021904701A8F9F7F1FE79
:10E10000F4E7052805D00DF5017DBDE83040F8F7AE
:10E1100047BF0DF5017D30BD74030300024B1B7832
:10E120000BB1FFF7D1BF70475743002030B505460C
:10E1300085B00C46002900F0A4800023CDE901330E
:10E14000514A039301230A608DF804008DF80630CC
:10E1500001A906232020ADF80830FFF7B1FF60B118
:10E16000F9F710FF494B4A4902464A481B1ADB0897
:10E170001B0443F00100F8F727FC0023CDE901332D
:10E1800003932268012301A940208DF80530FFF791
:10E1900097FF60B1F9F7F6FE3C4B3F4902463D4818
:10E1A0001B1ADB081B0443F00100F8F70DFC0023E9
:10E1B000CDE90133039322688DF80450F72301A9B8
:10E1C0002320ADF80630FFF77BFF60B1F9F7DAFEE8
:10E1D0002E4B324902462F481B1ADB081B0443F022
:10E1E0000100F8F7F1FB002301202268039301A945
:10E1F000CDE901338DF80400FFF762FF60B1F9F754
:10E20000C1FE224B2649024622481B1ADB081B048A
:10E2100043F00100F8F7D8FB0023CDE90233226870
:10E220004FF4B06301A9A1200193FFF749FF60B14A
:10E23000F9F7A8FE154B1B49024616481B1ADB08C6
:10E240001B0443F00100F8F7BFFB0025226803958B
:10E2500001A9A020CDE90155FFF732FF034668B1BF
:10E26000F9F790FE094B104902460A481B1ADB08D1
:10E270001B0443F00100F8F7A7FB2B46184605B036
:10E2800030BD0E23FAE700BFD82A0020B8EB020009
:10E29000F800030028EB02003E0103008A0103009E
:10E2A000D10103001D0203006E02030073B5054691
:10E2B0000668FFF703FF2B68B34204461DD91A48CE
:10E2C0001A4B1B491B1ADB081B0443F00200019088
:10E2D000F8F776FB2B68174901983246F8F77DFB73
:10E2E0004FF080532A68D3F80C31134901989B02F0
:10E2F00003F100539A1AF8F767FB2CB90F4B012270
:10E300001A70204602B070BD2046F9F73BFE074B5D
:10E310000B49024604481B1ADB081B0443F00100AA
:10E32000F8F752FBEDE700BF28EB0200B8EB020064
:10E33000C1020300F0020300210303005743002041
:10E340004B0303004BDF70471FB50E4C01A8FFF7CE
:10E35000F9FF70B9214602A8F9F7B9FD039B002B1C
:10E36000F4D00198D3E90021904702A8F9F7B9FD4C
:10E37000F4E7052804D004B0BDE81040F8F710BE5B
:10E3800004B010BD8C03030030B591EA030F00F117
:10E390008480841A71EB030C05D2121953EB0C0321
:10E3A000001B71EB0C0140F2000CCFF6E07C1CEA84
:10E3B000430F54D0BCEB410F61D90C0DA4EB135E9D
:10E3C00031EA0C0141F4801133EA0C0343F4801369
:10E3D000DEF1200C2AD303FA0CF5401941F10001BB
:10E3E00022FA0EF5401923FA0EF5694112FA0CF2E1
:10E3F000CD0208D349085FEA30005FEA320228BF45
:10E4000042F001020134013C5FEA500C72F100421B
:10E4100050F1000051EB04514FF4001313EB410F86
:10E4200038BF30BD090D0905002030BDBEF1200EFA
:10E43000BEF1200F1ED223FA0EF5401941F1000162
:10E44000CEF1200C124218BF012203FA0CF52A4328
:10E45000CEE711EA5C0F04BF0020002130BD1CEAAA
:10E46000410F04BF01F00041002030BD01F0004128
:10E47000002030BD21F4801101EB045130BD004279
:10E4800018BF41F00101BCEB410F08BF30BD4FF098
:10E49000FE4141F47801002030BD83F00043841A2E
:10E4A00071EB030E07D28EF0004E001B71EB0E01D4
:10E4B000121953EB0E0340F2000CCFF6E07C1CEA7D
:10E4C000430FC6D0BCEB410F72D90C0DA4EB135E09
:10E4D000C90241EA5051C00241F00041DB0243EA67
:10E4E0005253D20243F00043DEF1200C41D312FA22
:10E4F0000CF522FA0EF203FA0CF542EA050218BFF7
:10E5000042F0010223FA0EF3801A9941E30AC4F3A0
:10E510000A0411F0404F03D418D0013C4000494197
:10E52000013C23D44205C00A40EA4150C90A51EADD
:10E53000C3715FEA500C72F1004250F1000051EBE0
:10E54000045130BD01002FD00020203C0029F9D01B
:10E55000B1FA81FCDCF1200E11FA0CF130FA0EF563
:10E5600010FA0CF02943A4EB0C04D9E70020D907DA
:10E5700030BDAEF1200EBEF1200F0DD2CEF1200C39
:10E5800003FA0CF533FA0EF32A4318BF43F00103E4
:10E59000C01A61F10001B9E721F00041C00A40EA68
:10E5A0004150C90A01EB045130BD0020002130BDAB
:10E5B000004218BF41F00101BCEB410F7FF467AF8F
:10E5C000BCEB430F3FF463AF30BD00BF83F00043AB
:10E5D000FFF7DABEF0B540F2FF7681EA030C16EAE7
:10E5E000115E1EBFB64516EA1355B5425AD021EA50
:10E5F000465141F48011A1FB024723EA465343F4FC
:10E600008013AE44A0FB03650CF0004C36197D412D
:10E61000A1FB034747F10003A0FB0217F619654170
:10E6200053F10003094218BF46F0010640F2FE74A0
:10E63000B3F5007F13D2AEF5806EA6452BD24CEA1F
:10E640000331280341EA155140EA165032034508C8
:10E6500072F1004250F1000051EB0E51F0BDAEF2EC
:10E66000FF3EA64517D24CEAC321E80241EA5551C4
:10E6700040EA5650F202450872F1004250F10000A3
:10E6800051EB0E51F0BD0CF0004141F0FE4141F460
:10E6900070010020F0BD1EEA0E0FF4D50CF0004111
:10E6A0000020F0BD16EA115F04BF01F00041002018
:10E6B000004218BF41F0010116EA135F04BF03F0E6
:10E6C00000430022124218BF43F0010306EA13542C
:10E6D000B44218BF9EEA060F03D00CF000410020A0
:10E6E000F0BD21F0004123F00043B1EB065F06D8F6
:10E6F000B3EB065F03D8002918BF002BC3D140F24B
:10E700000001C7F6F8710020F0BD00BFC1F30A5345
:10E7100040F21E42D21A0EDD202A0AD8CB0243EA6A
:10E72000505040F00040D04090EAE170B0EBE17012
:10E730007047002070474B00004218BF43F00103B0
:10E7400013F5001F88BF21F0004111F0004058BFB1
:10E750006FF00040704700BF0B0D40F21E42D21A0E
:10E7600009DBCB0243EA505040F00040202A28BF8A
:10E770002022D0407047490060EB0000704700BF86
:10E78000C0F3C75191B142004FEA40704FEAD20145
:10E790004FEA310101F16051B2F17F4F38BF70474C
:10E7A00001F1605118BF41F40021704710F00041A1
:10E7B0000020704753EA020C61D02DE9F04BB3FA08
:10E7C00083F51E0007BFB2FA82F502FA05F403FAD8
:10E7D00005F41646C5F120051EBF22FA05F73C4395
:10E7E000203556EA044C4FEA144418BF0134A346BE
:10E7F0004FF00009C846904271EB030C39D309422F
:10E8000007BFB0FA80F700FA07F6B1FA81F701FA0C
:10E8100007F6C7F120071EBF20FA07FC46EA0C06E0
:10E820002037B6FBFBFC7F1B103F07F01F04C4F131
:10E8300020060CFA04F42CFA06F644BF34460026EF
:10E84000202FA4BF2646002454EA060C08BF01244A
:10E8500018EB040849EB0609A4FB027CC01B06FB6D
:10E8600002CC04FB03CC71EB0C01904271EB030C66
:10E87000C5D20B46024649464046BDE8F08BB2FB86
:10E88000F3F200007F2805D8034B185C034B5B5C58
:10E890001840704700207047A403030024040300BD
:10E8A000A0F16103192B98BF20387047A0F14103F4
:10E8B000192B98BF203070477F2805D8034B185C70
:10E8C000034B5B5C1840704700207047A4030300B3
:10E8D00024040300A0F16103192B98BF203870476E
:10E8E000A0F14103192B98BF203070477F299ABFB0
:10E8F000017001206FF02E0070475AB10A787F2A0C
:10E900000AD800B10260002119605960501A18BF7E
:10E9100001207047002070476FF02E007047000004
:10E9200008B5034B5B689B681B68984708BD00BF30
:10E93000382B002008B50921FFF7F2FF08BD8446F7
:10E9400040EA010313F0030F18D18446202A0BD3A9
:10E950002DE9F007B1E8F807A0E8F807A2F12002D6
:10E96000202AF7D2BDE8F007042A07D351F8043B68
:10E9700040F8043BA2F10402042AF7D2002A05D091
:10E9800011F8013B00F8013B013AF9D160467047AC
:10E990008446002A2DD010F0030F04D000F8011B8C
:10E9A000013A26D0F7E7C9B241EA012141EA014123
:10E9B000202A12D3A2F120022DE9F0030B460C46C7
:10E9C0000D460E460F4688468946A0E8FA03203ACF
:10E9D000FBD2BDE8F00320320BD0042A05D340F867
:10E9E000041B043A05D0042AF9D200F8011B013AAD
:10E9F000FBD160467047024610F0030F16D111F0AC
:10EA0000030F13D12DE9F0004FF001374FF08033A1
:10EA100051F8044BA4EB070525EA04051D4002D17B
:10EA200042F8044BF4E7A1F10401F0BC11F8013BFA
:10EA300002F8013B002BF9D1704700F1010110F001
:10EA4000030F11D010F8012B002A23D010F0030F70
:10EA50000AD010F8012B002A1CD010F0030F03D0AD
:10EA600010F8012B002A15D02DE970004FF001326B
:10EA70004FF0803350F8044BA4EB020525EA04055F
:10EA80001D4000D1F6E7A0F1040070BC10F8012B86
:0AEA9000002AFBD1A0EB0100704743
:10EA9C000D950200000000000D9A0200000000001D
:10EAAC009DD5020000000000D5AE02000000000061
:10EABC0049D202004839002071D90200883D00205B
:10EACC0011D402000000000087DB02000C3E002085
:10EADC003DDC0200102B0020A1B102000000000060
:08EAEC0051930200000000003C
:10EAF4001995020000000000A99A0200000000001D
:10EB04001DE102000000000049E3020000000000D3
:10EB1400902B0020582C0020602C0020982B0020E3
:04EB240018000000D5
:10EB2800E4F4020000000000EAF402000000000023
:10EB380010F5020000000000F1F4020000000000DF
:10EB480000F502000000000004F5020000000000CB
:10EB58000AF5020000000000F5F4020000000000C1
:10EB6800FAF402000000000014F5020000000000A2
:10EB780035EC0200000003030CED02000000000069
:10EB880035ED020000000000AD00030000000000A9
:10EB9800DEF4020000000000A000030000000303F0
:10EBA80059F4020000000303C5000300000003033A
:10EBB800680303000000030380030300000003034D
:10EBC800A6ED020000000000BCED020000000000FD
:10EBD80008EC02000000000014EC0200EC2A0020FF
:10EBE8000000000000000000018E0200000000008C
:04EBF8000000000019
:10EBFC00000000000338FDD870470000D563020008
:10EC0C0041640200D16302007274745F6C6F675FC1
:10EC1C006261636B656E64004261636B656E647305
:10EC2C0020666C757368656400617070000000008C
:10EC3C00803000207F000000003100201B5B313B46
:10EC4C0033316D0025734C6F67732064726F707075
:10EC5C006564202825642925730D0A001B5B306D23
:10EC6C00002573003C25733E2025733A2000202597
:10EC7C0030327800202020007C002563001B5B31A3
:10EC8C003B33306D001B5B313B33326D001B5B3112
:10EC9C003B33336D001B5B313B33346D001B5B31FD
:10ECAC003B33356D001B5B313B33366D001B5B31E9
:10ECBC003B33376D007761726E696E6700696E6603
:10ECCC006F0064656275670068EC020089EC0200F5
:10ECDC0048EC020091EC020099EC0200A1EC02005D
:10ECEC00A9EC0200B1EC0200B9EC0200000000003B
:10ECFC0022ED0200C1EC0200C9EC0200CEEC0200D5
:10ED0C006170705F627574746F6E0000203100204A
:10ED1C00466174616C206572726F72005379737402
:10ED2C00656D207265736574006170705F74696DD8
:10ED3C006572000001000600000000005C3100203C
:10ED4C002970020052544320696E7374616E6365BE
:10ED5C0020616C726561647920696E697469616C9B
:10ED6C00697A65642E005254433A20696E6974695D
:10ED7C00616C697A65642E000000000000000000E0
:10ED8C00000000000338FDD8704730313233343581
:10ED9C00363738394142434445467077725F6D6768
:10EDAC006D740000ECEA0200ECEA020004000000C2
:10EDBC00736F72746C697374004E52465F53554393
:10EDCC0043455353004E52465F4552524F525F5388
:10EDDC0056435F48414E444C45525F4D495353494D
:10EDEC004E47004E52465F4552524F525F534F466C
:10EDFC00544445564943455F4E4F545F454E41423E
:10EE0C004C4544004E52465F4552524F525F494E5C
:10EE1C005445524E414C004E52465F4552524F5251
:10EE2C005F4E4F5F4D454D004E52465F4552524F1F
:10EE3C00525F4E4F545F464F554E44004E52465F04
:10EE4C004552524F525F4E4F545F535550504F5294
:10EE5C00544544004E52465F4552524F525F494E04
:10EE6C0056414C49445F504152414D004E52465F11
:10EE7C004552524F525F494E56414C49445F535490
:10EE8C00415445004E52465F4552524F525F494ED7
:10EE9C0056414C49445F4C454E475448004E5246EF
:10EEAC005F4552524F525F494E56414C49445F4662
:10EEBC004C414753004E52465F4552524F525F49A8
:10EECC004E56414C49445F44415441004E52465FBA
:10EEDC004552524F525F444154415F53495A450089
:10EEEC004E52465F4552524F525F54494D454F5515
:10EEFC0054004E52465F4552524F525F4E554C4C49
:10EF0C00004E52465F4552524F525F464F52424955
:10EF1C004444454E004E52465F4552524F525F4953
:10EF2C004E56414C49445F41444452004E52465F58
:10EF3C004552524F525F42555359004E52465F450F
:10EF4C0052524F525F434F4E4E5F434F554E5400FB
:10EF5C004E52465F4552524F525F5245534F555297
:10EF6C00434553004E52465F4552524F525F4D4FF0
:10EF7C0044554C455F4E4F545F494E495449414CA2
:10EF8C00495A4544004E52465F4552524F525F4DCE
:10EF9C00555445585F494E49545F4641494C454488
:10EFAC00004E52465F4552524F525F4D5554455894
:10EFBC005F4C4F434B5F4641494C4544004E5246D3
:10EFCC005F4552524F525F4D555445585F554E4C0C
:10EFDC004F434B5F4641494C4544004E52465F45BA
:10EFEC0052524F525F4D555445585F434F4E445FFC
:10EFFC00494E49545F4641494C4544004E52465F88
:10F00C004552524F525F4D4F44554C455F414C5207
:10F01C00454144595F494E495449414C495A45442C
:10F02C00004E52465F4552524F525F53544F52411D
:10F03C0047455F46554C4C004E52465F4552524F29
:10F04C00525F4150495F4E4F545F494D504C454DB6
:10F05C00454E544544004E52465F4552524F525F06
:10F06C00464541545552455F4E4F545F454E4142C3
:10F07C004C4544004E52465F4552524F525F494FE9
:10F08C005F50454E44494E47004E52465F455252E2
:10F09C004F525F4452565F5457495F4552525F4F2F
:10F0AC0056455252554E004E52465F4552524F52A3
:10F0BC005F4452565F5457495F4552525F414E412F
:10F0CC00434B004E52465F4552524F525F4452568C
:10F0DC005F5457495F4552525F444E41434B004E7B
:10F0EC0052465F4552524F525F424C455F49505316
:10F0FC00505F52585F504B545F5452554E434154DD
:10F10C004544004E52465F4552524F525F424C4569
:10F11C005F495053505F4348414E4E454C5F414C04
:10F12C0052454144595F455849535453004E524639
:10F13C005F4552524F525F424C455F495053505FAE
:10F14C004C494E4B5F444953434F4E4E45435445F7
:10F15C0044004E52465F4552524F525F424C455FFF
:10F16C00495053505F504545525F52454A454354B0
:10F17C00454400556E6B6E6F776E206572726F72C0
:10F18C0020636F646500000000000000C5ED020004
:10F19C0001000000D1ED020002000000EFED0200C2
:10F1AC000300000010EE02000400000023EE020039
:10F1BC000500000034EE02000600000048EE0200DC
:10F1CC000700000060EE02000800000078EE02006C
:10F1DC000900000090EE02000A000000A9EE0200F7
:10F1EC000B000000C1EE02000C000000D8EE020083
:10F1FC000D000000ECEE02000E000000FEEE02001E
:10F20C000F0000000DEF02001000000021EF0200C3
:10F21C001100000038EF02001200000047EF02005E
:10F22C00130000005CEF02008000000070EF020091
:10F23C008100000091EF020082000000ADEF02009F
:10F24C0083000000C9EF020084000000E7EF020019
:10F25C008500000008F00200860000002DF002007E
:10F26C009000000044F002009100000062F00200E7
:10F27C009200000080F002000082000095F0020075
:10F28C0001820000B3F0020002820000CFF0020005
:10F29C0000840000EBF00200018400000FF102007A
:10F2AC000284000039F10200038400005EF10200C8
:10F2BC000000FFFFDEC0ADDEFE011EF1DEC0ADDEE4
:10F2CC00FF011EF1705F6673002573206368656330
:10F2DC006B206661696C656420696E202573282932
:10F2EC0020776974682076616C7565203078257894
:10F2FC002E00705F66732D3E705F61706900705FE9
:10F30C0064657374006C656E00616464725F69732C
:10F31C005F616C69676E65643332287372632900B0
:10F32C00616464725F69735F77697468696E5F6248
:10F33C006F756E647328705F66732C207372632C08
:10F34C00206C656E2900705F7372630021286C65F8
:10F35C006E202520705F66732D3E705F666C617346
:10F36C00685F696E666F2D3E70726F6772616D5F5C
:10F37C00756E69742900616464725F69735F616C96
:10F38C0069676E656433322864657374290061643F
:10F39C0064725F69735F616C69676E656433322890
:10F3AC002875696E7433325F7429705F73726329C8
:10F3BC0000616464725F69735F77697468696E5F1A
:10F3CC00626F756E647328705F66732C206465734E
:10F3DC00742C206C656E2900616464725F69735FC4
:10F3EC00706167655F616C69676E656428705F66E4
:10F3FC00732C20706167655F6164647229006164BD
:10F40C0064725F69735F77697468696E5F626F7548
:10F41C006E647328705F66732C20706167655F6122
:10F42C006464722C20286C656E202A20705F6673D1
:10F43C002D3E705F666C6173685F696E666F2D3E02
:10F44C0065726173655F756E69742929006E7266E9
:10F45C005F6673746F72616765006E72665F667368
:10F46C00746F726167655F6572617365006E726659
:10F47C005F6673746F726167655F7772697465003C
:10F48C006E72665F6673746F726167655F696E69D1
:10F49C0074000000001000000400000001000000D7
:10F4AC00959302007593020065930200A9950200E2
:10F4BC0059950200399302003D93020041930200DA
:10F4CC000000010100000001010000000D0E1112EE
:10F4DC001314636C6F636B00434C4F434B004750EA
:10F4EC00494F544500505253005541525400554118
:10F4FC005254450052544300534141444300544933
:10F50C004D45520050504900574454000D00030023
:10F51C0031AB02000E00030031AB0200F0340020CE
:10F52C0010350020303500204144433A25303464F6
:10F53C000D0A003C3C2020202020207764745F655D
:10F54C0076656E745F68616E646C65722829202024
:10F55C0020202020203E3E003D3D3E20416C69761F
:10F56C00652053656E64004576656E743A2025738C
:10F57C0020726563656976656420284E52465F5338
:10F58C0055434345535329004576656E743A2025FF
:10F59C00732072656365697665642028257329007C
:10F5AC005265636F72642049443A093078253034CF
:10F5BC00780046696C652049443A09307825303426
:10F5CC0078005265636F7264206B65793A09307804
:10F5DC002530347800424C455F4144565F455654C3
:10F5EC005F4641535400424C455F4144565F45567B
:10F5FC00545F49444C4500424C455F4741505F4580
:10F60C0056545F4144565F5245504F525420003C73
:10F61C003D3D3D3D3D3D3D3D3D3D3D3D20424C450F
:10F62C005F4741505F4556545F434F4E4E454354E0
:10F63C004544203D3D3D3D3D3D3D3D3D3E003C3D39
:10F64C003D3D3D3D3D3D3D3D3D3D3D20424C455FBD
:10F65C004741505F4556545F444953434F4E4E45C6
:10F66C0043544544203D3D3D3D3D3D3D3D3D3E00EB
:10F67C00424C455F4E55535F4556545F52585F445C
:10F68C00415441202841455329203D3E20003078EB
:10F69C00253032782C2000424C455F4E55535F4547
:10F6AC0056545F52585F4441544120284F524729C9
:10F6BC00203D3E2000424C455F4E55535F4556540D
:10F6CC005F54585F524459203D3D3D3D3D3D3E20E9
:10F6DC000A00424C455F4E55535F4556545F434FAD
:10F6EC004D4D5F53544152544544203D3D3D3D3DAD
:10F6FC003D3E200A00424C455F4E55535F455654E3
:10F70C005F434F4D4D5F53544F50504544203D3D4A
:10F71C003D3D3D3D3E200A0044617461206C656EA8
:10F72C002069732073657420746F203078255828F5
:10F73C0025642900566F6C3A2564202D2D205B25FD
:10F74C00645D0D0A004253505F4556454E545F4868
:10F75C00414E444C4552203D3E20256400404040E3
:10F76C0040404040204253505F4556454E545F4404
:10F77C0046553D3E256400404040404040402042BC
:10F78C0053505F4556454E545F414456455254497B
:10F79C0053494E475F53544152543D3E25640040FB
:10F7AC00404040404040204253505F4556454E54E7
:10F7BC005F4144564552544953494E475F53544F49
:10F7CC00503D3E2564004040404040404020627324
:10F7DC00705F6576656E745F68616E646C657228C7
:10F7EC0029202D2D20204253505F4556454E545F05
:10F7FC00534C45455000404040404040402042530F
:10F80C00505F4556454E545F57414B4555503D3E14
:10F81C002564006273705F6576656E745F68616EF7
:10F82C00646C65722829202D2D20204253505F4591
:10F83C0056454E545F444953434F4E4E4543540036
:10F84C006273705F6576656E745F68616E646C651B
:10F85C00722829202D2D20204253505F4556454EAD
:10F86C00545F57484954454C4953545F4F464600E2
:10F87C0053656E64456D6744617461282564290085
:10F88C0025303278200053656E645465737444617E
:10F89C00746128290053656E64416C697665446116
:10F8AC00746128290053656E645265674461746104
:10F8BC002829003D3D3D3E3E207469636B732069F1
:10F8CC0073205B25645D0053797374656D4D616EB7
:10F8DC00616765722E426C65436F6E6E656374650D
:10F8EC00643A25640A004D41432041646472657397
:10F8FC0073203A20253032582025303258202530BC
:10F90C003258000A3D3D3D3D3D3D3D3D3D3D3D3D7B
:10F91C003D3D3D3D3D3D3D3D3D3D3D3D3D3D3D3D0B
:10F92C003D3D3D3D3D3D3D3D3D3D3D3D3D3D3D3DFB
:10F93C003D3D3D3D3D3D3D3D3D3D3D3D3D3D3D0A1E
:10F94C000A004943532D323030422050726F677297
:10F95C00616D205374617274202D2D2D20566572AB
:10F96C0020312E313020323032322F30342F30349F
:10F97C00004465627567206C6F6767696E67206607
:10F98C006F722055415254206F7665722052545438
:10F99C0020737461727465642E004644535F45563F
:10F9AC00545F494E4954004644535F4556545F5783
:10F9BC0052495445004644535F4556545F55504494
:10F9CC00415445004644535F4556545F44454C5F93
:10F9DC005245434F5244004644535F4556545F448E
:10F9EC00454C5F46494C45004644535F4556545F71
:10F9FC00474300000000000002000003000000006C
:10FA0C0007000000FFFFFFFF0000000001000000E6
:10FA1C007201000001000000005C260506000000D9
:10FA2C00E83D002068FA020001000600000000001A
:10FA3C00000000000338FDD870470000A6F9020052
:10FA4C00B3F90200C1F90200D0F90200E3F9020097
:10FA5C00F4F90200A03D0020C83D002000900040B9
:10FA6C0000040000303E00205765734465637279D2
:10FA7C0070744563622041455331323800536D61D7
:10FA8C00727442616E6450415254524F4E0046445F
:10FA9C00535F4552525F4F5045524154494F4E5F50
:10FAAC0054494D454F5554004644535F4552525F9F
:10FABC004E4F545F494E495449414C495A454400B4
:10FACC004644535F4552525F554E414C49474E4553
:10FADC00445F41444452004644535F4552525F498F
:10FAEC004E56414C49445F415247004644535F4592
:10FAFC0052525F4E554C4C5F415247004644535F47
:10FB0C004552525F4E4F5F4F50454E5F5245434FEB
:10FB1C00524453004644535F4552525F4E4F5F531D
:10FB2C00504143455F494E5F464C41534800464463
:10FB3C00535F4552525F4E4F5F53504143455F49AF
:10FB4C004E5F515545554553004644535F455252FF
:10FB5C005F5245434F52445F544F4F5F4C415247A5
:10FB6C0045004644535F4552525F4E4F545F464FDB
:10FB7C00554E44004644535F4552525F4E4F5F50C2
:10FB8C0041474553004644535F4552525F555345D8
:10FB9C00525F4C494D49545F5245414348454400DE
:10FBAC004644535F4552525F4352435F434845437B
:10FBBC004B5F4641494C4544004644535F455252C5
:10FBCC005F42555359004644535F4552525F494E6C
:10FBDC005445524E414C00009AFA0200B4FA02000D
:10FBEC00CCFA0200E3FA0200F7FA020008FB02006A
:10FBFC0020FB02003AFB020055FB02006EFB0200E8
:10FC0C0080FB020091FB0200ACFB0200C5FB020072
:10FC1C00D2FB02002320454D47205072657373655B
:10FC2C00640023205465737420507265737365648B
:10FC3C0000232044657652656720507265737365A6
:10FC4C0064008D01020408102040801B366CD8AB78
:10FC5C004D9A2F5EBC63C697356AD4B37DFAEFC557
:10FC6C00913972E4D3BD61C29F254A943366CC832B
:10FC7C001D3A74E8CB8D01020408102040801B361D
:10FC8C006CD8AB4D9A2F5EBC63C697356AD4B37DE6
:10FC9C00FAEFC5913972E4D3BD61C29F254A943302
:10FCAC0066CC831D3A74E8CB8D0102040810204009
:10FCBC00801B366CD8AB4D9A2F5EBC63C697356AE9
:10FCCC00D4B37DFAEFC5913972E4D3BD61C29F25DF
:10FCDC004A943366CC831D3A74E8CB8D0102040838
:10FCEC00102040801B366CD8AB4D9A2F5EBC63C67F
:10FCFC0097356AD4B37DFAEFC5913972E4D3BD61FF
:10FD0C00C29F254A943366CC831D3A74E8CB8D018F
:10FD1C00020408102040801B366CD8AB4D9A2F5E25
:10FD2C00BC63C697356AD4B37DFAEFC5913972E4DA
:10FD3C00D3BD61C29F254A943366CC831D3A74E8C7
:10FD4C00CB52096AD53036A538BF40A39E81F3D774
:10FD5C00FB7CE339829B2FFF87348E4344C4DEE95E
:10FD6C00CB547B9432A6C2233DEE4C950B42FAC386
:10FD7C004E082EA16628D924B2765BA2496D8BD190
:10FD8C002572F8F66486689816D4A45CCC5D65B6CA
:10FD9C00926C704850FDEDB9DA5E154657A78D9DF3
:10FDAC008490D8AB008CBCD30AF7E45805B8B345A3
:10FDBC0006D02C1E8FCA3F0F02C1AFBD0301138AA0
:10FDCC006B3A9111414F67DCEA97F2CFCEF0B4E673
:10FDDC007396AC7422E7AD3585E2F937E81C75DF14
:10FDEC006E47F11A711D29C5896FB7620EAA18BE2C
:10FDFC001BFC563E4BC6D279209ADBC0FE78CD5AFE
:10FE0C00F41FDDA8338807C731B11210592780ECD5
:10FE1C005F60517FA919B54A0D2DE57A9F93C99C56
:10FE2C00EFA0E03B4DAE2AF5B0C8EBBB3C83539939
:10FE3C0061172B047EBA77D626E169146355210C21
:10FE4C007D637C777BF26B6FC53001672BFED7AB84
:10FE5C0076CA82C97DFA5947F0ADD4A2AF9CA47280
:10FE6C00C0B7FD9326363FF7CC34A5E5F171D831F8
:10FE7C001504C723C31896059A071280E2EB27B224
:10FE8C007509832C1A1B6E5AA0523BD6B329E32F4B
:10FE9C008453D100ED20FCB15B6ACBBE394A4C587F
:10FEAC00CFD0EFAAFB434D338545F9027F503C9FE1
:10FEBC00A851A3408F929D38F5BCB6DA2110FFF300
:10FECC00D2CD0C13EC5F974417C4A77E3D645D192B
:10FEDC007360814FDC222A908846EEB814DE5E0BEC
:10FEEC00DBE0323A0A4906245CC2D3AC629195E459
:10FEFC0079E7C8376D8DD54EA96C56F4EA657AAEA4
:10FF0C0008BA78252E1CA6B4C6E8DD741F4BBD8B31
:10FF1C008A703EB5664803F60E613557B986C11D29
:10FF2C009EE1F8981169D98E949B1E87E9CE5528CD
:10FF3C00DF8CA1890DBFE6426841992D0FB054BBEF
:10FF4C00165465726D696E616C00525454005345C1
:10FF5C00474745520073645F626C655F6761705F11
:10FF6C00646174615F6C656E6774685F7570646101
:10FF7C007465282920287265717565737429206F42
:10FF8C006E20636F6E6E656374696F6E20307825BA
:10FF9C00782072657475726E65642025732E00541A
:10FFAC006865207265717565737465642054582F8B
:10FFBC005258207061636B6574206C656E67746851
:10FFCC0020697320746F6F206C6F6E6720627920CC
:10FFDC0025752F2575206F63746574732E00546816
:10FFEC00652072657175657374656420636F6D62ED
:04FFFC00696E617455
:020000023000CC
:10000000696F6E206F6620545820616E64205258CC
:10001000207061636B6574206C656E677468732013
:10002000697320746F6F206C6F6E67206279202572
:1000300075206D6963726F7365636F6E64732E00F4
:1000400073645F626C655F67617474635F65786336
:1000500068616E67655F6D74755F726571756573F4
:100060007428292072657475726E65642025732E5C
:100070000073645F626C655F67617474735F657859
:100080006368616E67655F6D74755F7265706C79CA
:1000900028292072657475726E65642025732E00A0
:1000A0006E72665F626C655F6761747400626C6536
:1000B0005F6E7573009ECADC240EE5A9E093F3A37E
:1000C000B50000406E6E72665F73646800010000E8
:1000D00007000000ECEA0200F4EA02000800000059
:1000E00004EB020014EB020008000000F4EA020036
:1000F00004EB02000800000073645F626C655F63DC
:1001000066675F73657428292072657475726E6501
:1001100064202573207768656E20617474656D7046
:1001200074696E6720746F2073657420424C455F5C
:10013000434F4E4E5F4346475F4741502E00736426
:100140005F626C655F6366675F7365742829207200
:10015000657475726E6564202573207768656E20FE
:10016000617474656D7074696E6720746F20736557
:100170007420424C455F4741505F4346475F524FB2
:100180004C455F434F554E542E0073645F626C655F
:100190005F6366675F736574282920726574757282
:1001A0006E6564202573207768656E2061747465C0
:1001B0006D7074696E6720746F2073657420424C93
:1001C000455F434F4E4E5F4346475F474154542E71
:1001D0000073645F626C655F6366675F7365742854
:1001E000292072657475726E6564202573207768A6
:1001F000656E20617474656D7074696E6720746FCC
:100200002073657420424C455F434F4D4D4F4E5F08
:100210004346475F56535F555549442E0073645F0C
:10022000626C655F6366675F736574282920726519
:100230007475726E6564202573207768656E206121
:100240007474656D7074696E6720746F2073657463
:1002500020424C455F47415454535F4346475F41FA
:100260005454525F5441425F53495A452E007364BF
:100270005F626C655F6366675F73657428292072CF
:10028000657475726E6564202573207768656E20CD
:10029000617474656D7074696E6720746F20736526
:1002A0007420424C455F47415454535F4346475F77
:1002B000534552564943455F4348414E4745442EB6
:1002C00000496E73756666696369656E7420524194
:1002D0004D20616C6C6F636174656420666F722081
:1002E00074686520536F66744465766963652E0093
:1002F0004368616E6765207468652052414D2073C4
:1003000074617274206C6F636174696F6E206672C1
:100310006F6D203078257820746F20307825782E06
:10032000004D6178696D756D2052414D2073697A79
:100330006520666F72206170706C69636174696FAB
:100340006E20697320307825782E0073645F626CAC
:10035000655F656E61626C652829207265747572CF
:100360006E65642025732E006E72665F7364685F2D
:10037000626C6500ACEA0200ECEA020008000000D2
:100380006E72665F7364685F736F63009CEA02005D
:10039000ACEA02000800000043000000504F53493F
:1003A000580000002020202020202020206828281D
:1003B000282820202020202020202020202020202D
:1003C00020202020481010101010101010101010B5
:1003D0001010101084848484848484848484101095
:1003E00010101010108181818181810101010101B2
:1003F00001010101010101010101010101010110DE
:100400001010101010828282828282020202020286
:1004100002020202020202020202020202020210AE
:100420001010102000070320041702010857104085
:1004300080000000980303009C040300B005030043
:1004400053756E004D6F6E005475650057656400FE
:100450005468750046726900536174000000000022
:100460004A616E00466562004D6172004170720023
:100470004D6179004A756E004A756C0041756700E0
:10048000536570004F6374004E6F760044656300DF
:1004900000000000414D00504D000000D405030055
:1004A000D0050300D0050300D0050300D0050300EC
:1004B000D0050300D0050300D0050300D0050300DC
:1004C000D0050300FFFFFFFFFFFFFFFFFFFFFFFF60
:1004D000FFFF000010050300400403004C0503006B
:1004E0006004030094040300F4040300A405030063
:1004F00000050300256D2F25642F257900000000DD
:1005000025612025622025652025542025590000DD
:1005100053756E646179004D6F6E64617900547536
:100520006573646179005765646E65736461790011
:100530005468757273646179004672696461790008
:100540005361747572646179000000004A616E75D0
:10055000617279004665627275617279004D6172EF
:10056000636800417072696C004D6179004A756E74
:1005700065004A756C790041756775737400536541
:100580007074656D626572004F63746F62657200AE
:100590004E6F76656D62657200446563656D626578
:1005A0007200000025483A254D3A2553000000000E
:1005B00085E80200A1E80200ADE80200B9E8020007
:1005C000D5E80200E1E80200EDE80200FBE80200E5
:0605D000000000002E00F7
:1005D80000000000FF0000000010014011000400AE
:1005E8000090D0034943535745534433C0FFFFFF9E
:1005F8001400FFFF000000000000000000000000E1
:1006080000000000000000002C2B0020000000006B
:10061800C03D0020010004000D0E0000340403005A
:1006280034040300340403003404030034040300D6
:040000032000637501
:00000001FF
